 linkdata_support

 Timestamp is 5c762249 (Wed Feb 27 12:38:17 2019)

 Preferred load address is 10000000

 Start         Length     Name                   Class
 0001:00000000 000005e4H .text$di                CODE
 0001:000005f0 00002e5eH .text$mn                CODE
 0001:00003450 00000566H .text$x                 CODE
 0001:000039c0 0000019aH .text$yd                CODE
 0002:00000000 00000218H .idata$5                DATA
 0002:00000218 00000004H .CRT$XCA                DATA
 0002:0000021c 00000048H .CRT$XCU                DATA
 0002:00000264 00000004H .CRT$XCZ                DATA
 0002:00000268 00000004H .CRT$XIA                DATA
 0002:0000026c 00000004H .CRT$XIAA               DATA
 0002:00000270 00000004H .CRT$XIC                DATA
 0002:00000274 00000004H .CRT$XIZ                DATA
 0002:00000280 00000ec8H .rdata                  DATA
 0002:00001148 00000078H .rdata$debug            DATA
 0002:000011c0 00000304H .rdata$r                DATA
 0002:000014d0 00000058H .rdata$sxdata           DATA
 0002:00001528 00000004H .rtc$IAA                DATA
 0002:0000152c 00000004H .rtc$IZZ                DATA
 0002:00001530 00000004H .rtc$TAA                DATA
 0002:00001534 00000004H .rtc$TZZ                DATA
 0002:00001538 0000068cH .xdata$x                DATA
 0002:00001bd0 00000059H .edata                  DATA
 0002:00001c2c 000000a0H .idata$2                DATA
 0002:00001ccc 00000014H .idata$3                DATA
 0002:00001ce0 00000218H .idata$4                DATA
 0002:00001ef8 00001232H .idata$6                DATA
 0003:00000000 00000054H .data                   DATA
 0003:00000054 00000190H .data$r                 DATA
 0003:000001e8 000003b4H .bss                    DATA
 0004:00000000 00000058H .rsrc$01                DATA
 0004:00000060 00000180H .rsrc$02                DATA

  Address         Publics by Value              Rva+Base       Lib:Object

 0000:00000000       __except_list              00000000     <absolute>
 0000:00000000       ___guard_fids_count        00000000     <absolute>
 0000:00000000       ___guard_flags             00000000     <absolute>
 0000:00000000       ___guard_fids_table        00000000     <absolute>
 0000:00000016       ___safe_se_handler_count   00000016     <absolute>
 0000:00009876       __fltused                  00009876     <absolute>
 0000:00009876       __ldused                   00009876     <absolute>
 0000:00000000       ___ImageBase               10000000     <linker-defined>
 0001:000005f0       ??$_Allocate@D@std@@YAPADIPAD@Z 100015f0 f i LinkDataScriptLibrary.obj
 0001:00000620       ??$addressof@D@std@@YAPADAAD@Z 10001620 f i LinkDataScriptLibrary.obj
 0001:00000630       ??$construct@PADAAPAD@?$_Wrap_alloc@V?$allocator@D@std@@@std@@QAEXPAPADAAPAD@Z 10001630 f i LinkDataScriptLibrary.obj
 0001:00000650       ??$construct@PADAAPAD@?$allocator@D@std@@QAEXPAPADAAPAD@Z 10001650 f i LinkDataScriptLibrary.obj
 0001:00000670       ??$construct@PADAAPAD@?$allocator_traits@V?$allocator@D@std@@@std@@SAXAAV?$allocator@D@1@PAPADAAPAD@Z 10001670 f i LinkDataScriptLibrary.obj
 0001:00000690       ??$destroy@PAD@?$_Wrap_alloc@V?$allocator@D@std@@@std@@QAEXPAPAD@Z 10001690 f i LinkDataScriptLibrary.obj
 0001:000006a0       ??$destroy@PAD@?$allocator@D@std@@QAEXPAPAD@Z 100016a0 f i LinkDataScriptLibrary.obj
 0001:000006b0       ??$destroy@PAD@?$allocator_traits@V?$allocator@D@std@@@std@@SAXAAV?$allocator@D@1@PAPAD@Z 100016b0 f i LinkDataScriptLibrary.obj
 0001:000006c0       ??$forward@AAPAD@std@@YAAAPADAAPAD@Z 100016c0 f i LinkDataScriptLibrary.obj
 0001:000006d0       ??0?$QFlags@W4OpenModeFlag@QIODevice@@@@QAE@VQFlag@@@Z 100016d0 f i LinkDataScriptLibrary.obj
 0001:000006e0       ??0?$QFlags@W4OpenModeFlag@QIODevice@@@@QAE@W4OpenModeFlag@QIODevice@@@Z 100016e0 f i LinkDataScriptLibrary.obj
 0001:000006f0       ??0?$QFlags@W4ProcessEventsFlag@QEventLoop@@@@QAE@W4ProcessEventsFlag@QEventLoop@@@Z 100016f0 f i LinkDataScriptLibrary.obj
 0001:00000700       ??0?$QFlags@W4PropertyFlag@QScriptValue@@@@QAE@W4PropertyFlag@QScriptValue@@@Z 10001700 f i LinkDataScriptLibrary.obj
 0001:00000710       ??0?$_String_alloc@$0A@U?$_String_base_types@DV?$allocator@D@std@@@std@@@std@@QAE@ABV?$allocator@D@1@@Z 10001710 f i LinkDataScriptLibrary.obj
 0001:00000730       ??0?$_String_val@U?$_Simple_types@D@std@@@std@@QAE@XZ 10001730 f i LinkDataScriptLibrary.obj
 0001:00000750       ??0?$_Wrap_alloc@V?$allocator@D@std@@@std@@QAE@XZ 10001750 f i LinkDataScriptLibrary.obj
 0001:00000760       ??0?$allocator@D@std@@QAE@XZ 10001760 f i LinkDataScriptLibrary.obj
 0001:00000770       ??0?$basic_string@DU?$char_traits@D@std@@V?$allocator@D@2@@std@@QAE@PBD@Z 10001770 f i LinkDataScriptLibrary.obj
 0001:000007d0       ??0LinkDataRequestHandler@U2@@QAE@PAVQEventLoop@@@Z 100017d0 f   LinkDataScriptLibrary.obj
 0001:00000850       ??0QFlag@@QAE@H@Z          10001850 f i LinkDataScriptLibrary.obj
 0001:00000860       ??0QLatin1Char@@QAE@D@Z    10001860 f i LinkDataScriptLibrary.obj
 0001:00000870       ??0_Generic_error_category@std@@QAE@XZ 10001870 f i LinkDataScriptLibrary.obj
 0001:00000880       ??0_Ignore@std@@QAE@XZ     10001880 f i LinkDataScriptLibrary.obj
 0001:00000890       ??0_Iostream_error_category@std@@QAE@XZ 10001890 f i LinkDataScriptLibrary.obj
 0001:000008a0       ??0_System_error_category@std@@QAE@XZ 100018a0 f i LinkDataScriptLibrary.obj
 0001:000008b0       ??0error_category@std@@QAE@XZ 100018b0 f i LinkDataScriptLibrary.obj
 0001:000008c0       ??0error_condition@std@@QAE@HABVerror_category@1@@Z 100018c0 f i LinkDataScriptLibrary.obj
 0001:000008e0       ??1?$basic_string@DU?$char_traits@D@std@@V?$allocator@D@2@@std@@QAE@XZ 100018e0 f i LinkDataScriptLibrary.obj
 0001:00000910       ??1LinkDataRequestHandler@U2@@UAE@XZ 10001910 f i LinkDataScriptLibrary.obj
 0001:00000980       ??1_Generic_error_category@std@@UAE@XZ 10001980 f i LinkDataScriptLibrary.obj
 0001:00000990       ??1_Iostream_error_category@std@@UAE@XZ 10001990 f i LinkDataScriptLibrary.obj
 0001:000009a0       ??1_System_error_category@std@@UAE@XZ 100019a0 f i LinkDataScriptLibrary.obj
 0001:000009b0       ??1error_category@std@@UAE@XZ 100019b0 f i LinkDataScriptLibrary.obj
 0001:000009c0       ??2@YAPAXIPAX@Z            100019c0 f i LinkDataScriptLibrary.obj
 0001:000009d0       ??3@YAXPAX0@Z              100019d0 f i LinkDataScriptLibrary.obj
 0001:000009e0       ??8error_category@std@@QBE_NABV01@@Z 100019e0 f i LinkDataScriptLibrary.obj
 0001:000009f0       ??8error_condition@std@@QBE_NABV01@@Z 100019f0 f i LinkDataScriptLibrary.obj
 0001:00000a10       ??BQFlag@@QBEHXZ           10001a10 f i LinkDataScriptLibrary.obj
 0001:00000a20       ??H@YA?BVQByteArray@@ABV0@PBD@Z 10001a20 f i LinkDataScriptLibrary.obj
 0001:00000aa0       ??H@YA?BVQByteArray@@PBDABV0@@Z 10001aa0 f i LinkDataScriptLibrary.obj
 0001:00000b20       ??U?$QFlags@W4OpenModeFlag@QIODevice@@@@QBE?AV0@W4OpenModeFlag@QIODevice@@@Z 10001b20 f i LinkDataScriptLibrary.obj
 0001:00000b40       ??U@YA?AV?$QFlags@W4OpenModeFlag@QIODevice@@@@W4OpenModeFlag@QIODevice@@0@Z 10001b40 f i LinkDataScriptLibrary.obj
 0001:00000b50       ??_GLinkDataRequestHandler@U2@@UAEPAXI@Z 10001b50 f i LinkDataScriptLibrary.obj
 0001:00000b50       ??_ELinkDataRequestHandler@U2@@UAEPAXI@Z 10001b50 f i LinkDataScriptLibrary.obj
 0001:00000bd0       ??_E_Generic_error_category@std@@UAEPAXI@Z 10001bd0 f i LinkDataScriptLibrary.obj
 0001:00000bd0       ??_G_Generic_error_category@std@@UAEPAXI@Z 10001bd0 f i LinkDataScriptLibrary.obj
 0001:00000c00       ??_E_Iostream_error_category@std@@UAEPAXI@Z 10001c00 f i LinkDataScriptLibrary.obj
 0001:00000c00       ??_G_Iostream_error_category@std@@UAEPAXI@Z 10001c00 f i LinkDataScriptLibrary.obj
 0001:00000c30       ??_E_System_error_category@std@@UAEPAXI@Z 10001c30 f i LinkDataScriptLibrary.obj
 0001:00000c30       ??_G_System_error_category@std@@UAEPAXI@Z 10001c30 f i LinkDataScriptLibrary.obj
 0001:00000c60       ??_Gerror_category@std@@UAEPAXI@Z 10001c60 f i LinkDataScriptLibrary.obj
 0001:00000c60       ??_Eerror_category@std@@UAEPAXI@Z 10001c60 f i LinkDataScriptLibrary.obj
 0001:00000c90       ?_Copy@?$basic_string@DU?$char_traits@D@std@@V?$allocator@D@2@@std@@QAEXII@Z 10001c90 f i LinkDataScriptLibrary.obj
 0001:00000de0       ?_Eos@?$basic_string@DU?$char_traits@D@std@@V?$allocator@D@2@@std@@QAEXI@Z 10001de0 f i LinkDataScriptLibrary.obj
 0001:00000e10       ?_Getal@?$_String_alloc@$0A@U?$_String_base_types@DV?$allocator@D@std@@@std@@@std@@QBE?AU?$_Wrap_alloc@V?$allocator@D@std@@@2@XZ 10001e10 f i LinkDataScriptLibrary.obj
 0001:00000e20       ?_Grow@?$basic_string@DU?$char_traits@D@std@@V?$allocator@D@2@@std@@QAE_NI_N@Z 10001e20 f i LinkDataScriptLibrary.obj
 0001:00000ed0       ?_Inside@?$basic_string@DU?$char_traits@D@std@@V?$allocator@D@2@@std@@QAE_NPBD@Z 10001ed0 f i LinkDataScriptLibrary.obj
 0001:00000f10       ?_Myptr@?$_String_val@U?$_Simple_types@D@std@@@std@@QAEPADXZ 10001f10 f i LinkDataScriptLibrary.obj
 0001:00000f20       ?_Myptr@?$_String_val@U?$_Simple_types@D@std@@@std@@QBEPBDXZ 10001f20 f i LinkDataScriptLibrary.obj
 0001:00000f30       ?_Tidy@?$basic_string@DU?$char_traits@D@std@@V?$allocator@D@2@@std@@QAEX_NI@Z 10001f30 f i LinkDataScriptLibrary.obj
 0001:00000f80       ?_Xlen@?$basic_string@DU?$char_traits@D@std@@V?$allocator@D@2@@std@@QBEXXZ 10001f80 f i LinkDataScriptLibrary.obj
 0001:00000f90       ?_Xran@?$basic_string@DU?$char_traits@D@std@@V?$allocator@D@2@@std@@QBEXXZ 10001f90 f i LinkDataScriptLibrary.obj
 0001:00000fa0       ?allocate@?$_Wrap_alloc@V?$allocator@D@std@@@std@@QAEPADI@Z 10001fa0 f i LinkDataScriptLibrary.obj
 0001:00000fd0       ?allocate@?$allocator@D@std@@QAEPADI@Z 10001fd0 f i LinkDataScriptLibrary.obj
 0001:00001000       ?assign@?$basic_string@DU?$char_traits@D@std@@V?$allocator@D@2@@std@@QAEAAV12@ABV12@II@Z 10002000 f i LinkDataScriptLibrary.obj
 0001:00001120       ?assign@?$basic_string@DU?$char_traits@D@std@@V?$allocator@D@2@@std@@QAEAAV12@PBD@Z 10002120 f i LinkDataScriptLibrary.obj
 0001:00001160       ?assign@?$basic_string@DU?$char_traits@D@std@@V?$allocator@D@2@@std@@QAEAAV12@PBDI@Z 10002160 f i LinkDataScriptLibrary.obj
 0001:00001260       ?assign@?$char_traits@D@std@@SAXAADABD@Z 10002260 f i LinkDataScriptLibrary.obj
 0001:00001270       ?category@error_code@std@@QBEABVerror_category@2@XZ 10002270 f i LinkDataScriptLibrary.obj
 0001:00001280       ?category@error_condition@std@@QBEABVerror_category@2@XZ 10002280 f i LinkDataScriptLibrary.obj
 0001:00001290       ?copy@?$char_traits@D@std@@SAPADPADPBDI@Z 10002290 f i LinkDataScriptLibrary.obj
 0001:000012b0       ?deallocate@?$_Wrap_alloc@V?$allocator@D@std@@@std@@QAEXPADI@Z 100022b0 f i LinkDataScriptLibrary.obj
 0001:000012d0       ?deallocate@?$allocator@D@std@@QAEXPADI@Z 100022d0 f i LinkDataScriptLibrary.obj
 0001:000012f0       ?default_error_condition@_System_error_category@std@@UBE?AVerror_condition@2@H@Z 100022f0 f i LinkDataScriptLibrary.obj
 0001:00001330       ?default_error_condition@error_category@std@@UBE?AVerror_condition@2@H@Z 10002330 f i LinkDataScriptLibrary.obj
 0001:00001350       ?equivalent@error_category@std@@UBE_NABVerror_code@2@H@Z 10002350 f i LinkDataScriptLibrary.obj
 0001:00001370       ?equivalent@error_category@std@@UBE_NHABVerror_condition@2@@Z 10002370 f i LinkDataScriptLibrary.obj
 0001:000013b0       ?erase@?$basic_string@DU?$char_traits@D@std@@V?$allocator@D@2@@std@@QAEAAV12@I@Z 100023b0 f i LinkDataScriptLibrary.obj
 0001:000013f0       ?erase@?$basic_string@DU?$char_traits@D@std@@V?$allocator@D@2@@std@@QAEAAV12@II@Z 100023f0 f i LinkDataScriptLibrary.obj
 0001:00001490       ?errorString@LinkDataRequestHandler@U2@@QBE?BVQString@@XZ 10002490 f   LinkDataScriptLibrary.obj
 0001:000014c0       ?fetchFile@LinkDataScriptLibrary@U2@@SA?AVQScriptValue@@PAVQScriptContext@@PAVQScriptEngine@@@Z 100024c0 f   LinkDataScriptLibrary.obj
 0001:00001a60       ?generic_category@std@@YAABVerror_category@1@XZ 10002a60 f i LinkDataScriptLibrary.obj
 0001:00001a70       ?getResult@LinkDataRequestHandler@U2@@QBE?AVQByteArray@@XZ 10002a70 f   LinkDataScriptLibrary.obj
 0001:00001aa0       ?hasError@LinkDataRequestHandler@U2@@QBE_NXZ 10002aa0 f   LinkDataScriptLibrary.obj
 0001:00001ab0       ?init@LinkDataScriptLibrary@U2@@SAXPAVWorkflowScriptEngine@2@@Z 10002ab0 f   LinkDataScriptLibrary.obj
 0001:00001c80       ?length@?$char_traits@D@std@@SAIPBD@Z 10002c80 f i LinkDataScriptLibrary.obj
 0001:00001ca0       ?max_size@?$_Wrap_alloc@V?$allocator@D@std@@@std@@QBEIXZ 10002ca0 f i LinkDataScriptLibrary.obj
 0001:00001cb0       ?max_size@?$allocator@D@std@@QBEIXZ 10002cb0 f i LinkDataScriptLibrary.obj
 0001:00001cc0       ?max_size@?$allocator_traits@V?$allocator@D@std@@@std@@SAIABV?$allocator@D@2@@Z 10002cc0 f i LinkDataScriptLibrary.obj
 0001:00001cd0       ?max_size@?$basic_string@DU?$char_traits@D@std@@V?$allocator@D@2@@std@@QBEIXZ 10002cd0 f i LinkDataScriptLibrary.obj
 0001:00001ce0       ?message@_Generic_error_category@std@@UBE?AV?$basic_string@DU?$char_traits@D@std@@V?$allocator@D@2@@2@H@Z 10002ce0 f i LinkDataScriptLibrary.obj
 0001:00001d60       ?message@_Iostream_error_category@std@@UBE?AV?$basic_string@DU?$char_traits@D@std@@V?$allocator@D@2@@2@H@Z 10002d60 f i LinkDataScriptLibrary.obj
 0001:00001db0       ?message@_System_error_category@std@@UBE?AV?$basic_string@DU?$char_traits@D@std@@V?$allocator@D@2@@2@H@Z 10002db0 f i LinkDataScriptLibrary.obj
 0001:00001e30       ?move@?$char_traits@D@std@@SAPADPADPBDI@Z 10002e30 f i LinkDataScriptLibrary.obj
 0001:00001e50       ?name@_Generic_error_category@std@@UBEPBDXZ 10002e50 f i LinkDataScriptLibrary.obj
 0001:00001e60       ?name@_Iostream_error_category@std@@UBEPBDXZ 10002e60 f i LinkDataScriptLibrary.obj
 0001:00001e70       ?name@_System_error_category@std@@UBEPBDXZ 10002e70 f i LinkDataScriptLibrary.obj
 0001:00001e80       ?onProxyAuthenticationRequired@LinkDataRequestHandler@U2@@AAEXABVQNetworkProxy@@PAVQAuthenticator@@@Z 10002e80 f   LinkDataScriptLibrary.obj
 0001:00001ff0       ?size@?$basic_string@DU?$char_traits@D@std@@V?$allocator@D@2@@std@@QBEIXZ 10002ff0 f i LinkDataScriptLibrary.obj
 0001:00002000       ?sl_onReplyFinished@LinkDataRequestHandler@U2@@AAEXPAVQNetworkReply@@@Z 10003000 f   LinkDataScriptLibrary.obj
 0001:000020b0       ?system_category@std@@YAABVerror_category@1@XZ 100030b0 f i LinkDataScriptLibrary.obj
 0001:000020c0       ?tr@LinkDataRequestHandler@U2@@SA?AVQString@@PBD0H@Z 100030c0 f i LinkDataScriptLibrary.obj
 0001:000020f0       ?value@error_code@std@@QBEHXZ 100030f0 f i LinkDataScriptLibrary.obj
 0001:00002100       ?value@error_condition@std@@QBEHXZ 10003100 f i LinkDataScriptLibrary.obj
 0001:00002110       _hypot                     10003110 f i LinkDataScriptLibrary.obj
 0001:00002140       ??0LinkDataScriptFactory@U2@@QAE@XZ 10003140 f i LinkDataSupportPlugin.obj
 0001:00002150       ??0LinkDataSupportPlugin@U2@@QAE@XZ 10003150 f   LinkDataSupportPlugin.obj
 0001:00002220       ??1LinkDataScriptFactory@U2@@UAE@XZ 10003220 f i LinkDataSupportPlugin.obj
 0001:00002230       ??1LinkDataSupportPlugin@U2@@UAE@XZ 10003230 f i LinkDataSupportPlugin.obj
 0001:00002240       ??_ELinkDataScriptFactory@U2@@UAEPAXI@Z 10003240 f i LinkDataSupportPlugin.obj
 0001:00002240       ??_GLinkDataScriptFactory@U2@@UAEPAXI@Z 10003240 f i LinkDataSupportPlugin.obj
 0001:00002270       ??_GLinkDataSupportPlugin@U2@@UAEPAXI@Z 10003270 f i LinkDataSupportPlugin.obj
 0001:00002270       ??_ELinkDataSupportPlugin@U2@@UAEPAXI@Z 10003270 f i LinkDataSupportPlugin.obj
 0001:000022a0       ?createScript@LinkDataScriptFactory@U2@@UAEXPAVWorkflowScriptEngine@2@@Z 100032a0 f   LinkDataSupportPlugin.obj
 0001:000022c0       ?tr@LinkDataSupportPlugin@U2@@SA?AVQString@@PBD0H@Z 100032c0 f i LinkDataSupportPlugin.obj
 0001:000022f0       _ugene_plugin_init         100032f0 f   LinkDataSupportPlugin.obj
 0001:00002310       ??C?$QScopedPointer@VQObjectData@@U?$QScopedPointerDeleter@VQObjectData@@@@@@QBEPAVQObjectData@@XZ 10003310 f i moc_LinkDataScriptLibrary.obj
 0001:00002320       ?metaObject@LinkDataRequestHandler@U2@@UBEPBUQMetaObject@@XZ 10003320 f   moc_LinkDataScriptLibrary.obj
 0001:00002340       ?qt_metacall@LinkDataRequestHandler@U2@@UAEHW4Call@QMetaObject@@HPAPAX@Z 10003340 f   moc_LinkDataScriptLibrary.obj
 0001:000023b0       ?qt_metacast@LinkDataRequestHandler@U2@@UAEPAXPBD@Z 100033b0 f   moc_LinkDataScriptLibrary.obj
 0001:00002410       ?qt_noop@@YAXXZ            10003410 f i moc_LinkDataScriptLibrary.obj
 0001:00002420       ?qt_static_metacall@LinkDataRequestHandler@U2@@CAXPAVQObject@@W4Call@QMetaObject@@HPAPAX@Z 10003420 f   moc_LinkDataScriptLibrary.obj
 0001:00002460       ?metaObject@LinkDataSupportPlugin@U2@@UBEPBUQMetaObject@@XZ 10003460 f   moc_LinkDataSupportPlugin.obj
 0001:00002480       ?qt_metacall@LinkDataSupportPlugin@U2@@UAEHW4Call@QMetaObject@@HPAPAX@Z 10003480 f   moc_LinkDataSupportPlugin.obj
 0001:00002490       ?qt_metacast@LinkDataSupportPlugin@U2@@UAEPAXPBD@Z 10003490 f   moc_LinkDataSupportPlugin.obj
 0001:000024f0       ?qt_static_metacall@LinkDataSupportPlugin@U2@@CAXPAVQObject@@W4Call@QMetaObject@@HPAPAX@Z 100034f0 f   moc_LinkDataSupportPlugin.obj
 0001:00002500       ??0initializer@?A0x896ef0f2@@QAE@XZ 10003500 f i qrc_linkdata_support.obj
 0001:00002520       ??1initializer@?A0x896ef0f2@@QAE@XZ 10003520 f i qrc_linkdata_support.obj
 0001:00002540       ?qCleanupResources_linkdata_support@@YAHXZ 10003540 f   qrc_linkdata_support.obj
 0001:00002560       ?qInitResources_linkdata_support@@YAHXZ 10003560 f   qrc_linkdata_support.obj
 0001:00002580       ?getAppSettings@AppContext@U2@@SAPAVAppSettings@2@XZ 10003580 f   U2Core:U2Core.dll
 0001:00002586       ??0Logger@U2@@QAE@ABVQString@@@Z 10003586 f   U2Core:U2Core.dll
 0001:0000258c       ??1Logger@U2@@UAE@XZ       1000358c f   U2Core:U2Core.dll
 0001:00002592       ?trace@Logger@U2@@QAEXABVQString@@@Z 10003592 f   U2Core:U2Core.dll
 0001:00002598       ?getProxyByUrl@NetworkConfiguration@U2@@QBE?AVQNetworkProxy@@ABVQUrl@@@Z 10003598 f   U2Core:U2Core.dll
 0001:0000259e       ??0Plugin@U2@@QAE@ABVQString@@0_NW4PluginState@1@@Z 1000359e f   U2Core:U2Core.dll
 0001:000025a4       ??1Plugin@U2@@UAE@XZ       100035a4 f   U2Core:U2Core.dll
 0001:000025aa       ?getWorkflowScriptRegistry@AppContext@U2@@SAPAVWorkflowScriptRegistry@2@XZ 100035aa f   U2Core:U2Core.dll
 0001:000025b0       ?qt_metacast@Plugin@U2@@UAEPAXPBD@Z 100035b0 f   U2Core:U2Core.dll
 0001:000025b6       ?qt_metacall@Plugin@U2@@UAEHW4Call@QMetaObject@@HPAPAX@Z 100035b6 f   U2Core:U2Core.dll
 0001:000025bc       ??1WorkflowScriptFactory@U2@@UAE@XZ 100035bc f   U2Lang:U2Lang.dll
 0001:000025c2       ?registerScriptFactory@WorkflowScriptRegistry@U2@@QAEXPAVWorkflowScriptFactory@2@@Z 100035c2 f   U2Lang:U2Lang.dll
 0001:000025c8       ??1QScriptValue@@QAE@XZ    100035c8 f   Qt5Script:Qt5Script.dll
 0001:000025ce       ??0QScriptValue@@QAE@ABV0@@Z 100035ce f   Qt5Script:Qt5Script.dll
 0001:000025d4       ?isObject@QScriptValue@@QBE_NXZ 100035d4 f   Qt5Script:Qt5Script.dll
 0001:000025da       ?toString@QScriptValue@@QBE?AVQString@@XZ 100035da f   Qt5Script:Qt5Script.dll
 0001:000025e0       ?setProperty@QScriptValue@@QAEXABVQString@@ABV1@ABV?$QFlags@W4PropertyFlag@QScriptValue@@@@@Z 100035e0 f   Qt5Script:Qt5Script.dll
 0001:000025e6       ?argumentCount@QScriptContext@@QBEHXZ 100035e6 f   Qt5Script:Qt5Script.dll
 0001:000025ec       ?argument@QScriptContext@@QBE?AVQScriptValue@@H@Z 100035ec f   Qt5Script:Qt5Script.dll
 0001:000025f2       ?throwError@QScriptContext@@QAE?AVQScriptValue@@ABVQString@@@Z 100035f2 f   Qt5Script:Qt5Script.dll
 0001:000025f8       ?globalObject@QScriptEngine@@QBE?AVQScriptValue@@XZ 100035f8 f   Qt5Script:Qt5Script.dll
 0001:000025fe       ?evaluate@QScriptEngine@@QAE?AVQScriptValue@@ABVQString@@0H@Z 100035fe f   Qt5Script:Qt5Script.dll
 0001:00002604       ?newFunction@QScriptEngine@@QAE?AVQScriptValue@@P6A?AV2@PAVQScriptContext@@PAV1@@ZH@Z 10003604 f   Qt5Script:Qt5Script.dll
 0001:0000260a       ?newObject@QScriptEngine@@QAE?AVQScriptValue@@XZ 1000360a f   Qt5Script:Qt5Script.dll
 0001:00002610       ??0QNetworkRequest@@QAE@ABVQUrl@@@Z 10003610 f   Qt5Network:Qt5Network.dll
 0001:00002616       ??1QNetworkRequest@@QAE@XZ 10003616 f   Qt5Network:Qt5Network.dll
 0001:0000261c       ??0QNetworkAccessManager@@QAE@PAVQObject@@@Z 1000361c f   Qt5Network:Qt5Network.dll
 0001:00002622       ??1QNetworkAccessManager@@UAE@XZ 10003622 f   Qt5Network:Qt5Network.dll
 0001:00002628       ?setProxy@QNetworkAccessManager@@QAEXABVQNetworkProxy@@@Z 10003628 f   Qt5Network:Qt5Network.dll
 0001:0000262e       ?get@QNetworkAccessManager@@QAEPAVQNetworkReply@@ABVQNetworkRequest@@@Z 1000362e f   Qt5Network:Qt5Network.dll
 0001:00002634       ?error@QNetworkReply@@QBE?AW4NetworkError@1@XZ 10003634 f   Qt5Network:Qt5Network.dll
 0001:0000263a       ??1QNetworkProxy@@QAE@XZ   1000363a f   Qt5Network:Qt5Network.dll
 0001:00002640       ?user@QNetworkProxy@@QBE?AVQString@@XZ 10003640 f   Qt5Network:Qt5Network.dll
 0001:00002646       ?password@QNetworkProxy@@QBE?AVQString@@XZ 10003646 f   Qt5Network:Qt5Network.dll
 0001:0000264c       ?setUser@QAuthenticator@@QAEXABVQString@@@Z 1000364c f   Qt5Network:Qt5Network.dll
 0001:00002652       ?setPassword@QAuthenticator@@QAEXABVQString@@@Z 10003652 f   Qt5Network:Qt5Network.dll
 0001:00002658       ?tr@QMetaObject@@QBE?AVQString@@PBD0H@Z 10003658 f   Qt5Core:Qt5Core.dll
 0001:0000265e       ??1Connection@QMetaObject@@QAE@XZ 1000365e f   Qt5Core:Qt5Core.dll
 0001:00002664       ??0QChar@@QAE@UQLatin1Char@@@Z 10003664 f   Qt5Core:Qt5Core.dll
 0001:0000266a       ??0QByteArray@@QAE@XZ      1000366a f   Qt5Core:Qt5Core.dll
 0001:00002670       ??0QByteArray@@QAE@PBDH@Z  10003670 f   Qt5Core:Qt5Core.dll
 0001:00002676       ??0QByteArray@@QAE@ABV0@@Z 10003676 f   Qt5Core:Qt5Core.dll
 0001:0000267c       ??1QByteArray@@QAE@XZ      1000367c f   Qt5Core:Qt5Core.dll
 0001:00002682       ?append@QByteArray@@QAEAAV1@PBD@Z 10003682 f   Qt5Core:Qt5Core.dll
 0001:00002688       ?append@QByteArray@@QAEAAV1@ABV1@@Z 10003688 f   Qt5Core:Qt5Core.dll
 0001:0000268e       ??0QString@@QAE@XZ         1000368e f   Qt5Core:Qt5Core.dll
 0001:00002694       ??0QString@@QAE@ABV0@@Z    10003694 f   Qt5Core:Qt5Core.dll
 0001:0000269a       ??1QString@@QAE@XZ         1000369a f   Qt5Core:Qt5Core.dll
 0001:000026a0       ??4QString@@QAEAAV0@$$QAV0@@Z 100036a0 f   Qt5Core:Qt5Core.dll
 0001:000026a6       ?arg@QString@@QBE?AV1@ABV1@HVQChar@@@Z 100036a6 f   Qt5Core:Qt5Core.dll
 0001:000026ac       ??0QString@@QAE@ABVQByteArray@@@Z 100036ac f   Qt5Core:Qt5Core.dll
 0001:000026b2       ?isNull@QString@@QBE_NXZ   100036b2 f   Qt5Core:Qt5Core.dll
 0001:000026b8       ?fromAscii_helper@QString@@CAPAU?$QTypedArrayData@G@@PBDH@Z 100036b8 f   Qt5Core:Qt5Core.dll
 0001:000026be       ?tr@QObject@@SA?AVQString@@PBD0H@Z 100036be f   Qt5Core:Qt5Core.dll
 0001:000026c4       ??0QObject@@QAE@PAV0@@Z    100036c4 f   Qt5Core:Qt5Core.dll
 0001:000026ca       ??1QObject@@UAE@XZ         100036ca f   Qt5Core:Qt5Core.dll
 0001:000026d0       ?connect@QObject@@QBE?AVConnection@QMetaObject@@PBV1@PBD1W4ConnectionType@Qt@@@Z 100036d0 f   Qt5Core:Qt5Core.dll
 0001:000026d6       ?disconnect@QObject@@SA_NPBV1@PBD01@Z 100036d6 f   Qt5Core:Qt5Core.dll
 0001:000026dc       ??0QEventLoop@@QAE@PAVQObject@@@Z 100036dc f   Qt5Core:Qt5Core.dll
 0001:000026e2       ??1QEventLoop@@UAE@XZ      100036e2 f   Qt5Core:Qt5Core.dll
 0001:000026e8       ?exec@QEventLoop@@QAEHV?$QFlags@W4ProcessEventsFlag@QEventLoop@@@@@Z 100036e8 f   Qt5Core:Qt5Core.dll
 0001:000026ee       ?exit@QEventLoop@@QAEXH@Z  100036ee f   Qt5Core:Qt5Core.dll
 0001:000026f4       ?readAll@QIODevice@@QAE?AVQByteArray@@XZ 100036f4 f   Qt5Core:Qt5Core.dll
 0001:000026fa       ?errorString@QIODevice@@QBE?AVQString@@XZ 100036fa f   Qt5Core:Qt5Core.dll
 0001:00002700       ??0QUrl@@QAE@ABVQString@@W4ParsingMode@0@@Z 10003700 f   Qt5Core:Qt5Core.dll
 0001:00002706       ??1QUrl@@QAE@XZ            10003706 f   Qt5Core:Qt5Core.dll
 0001:0000270c       ??0QTextStream@@QAE@PAVQIODevice@@@Z 1000370c f   Qt5Core:Qt5Core.dll
 0001:00002712       ??1QTextStream@@UAE@XZ     10003712 f   Qt5Core:Qt5Core.dll
 0001:00002718       ?readAll@QTextStream@@QAE?AVQString@@XZ 10003718 f   Qt5Core:Qt5Core.dll
 0001:0000271e       ??0QFile@@QAE@ABVQString@@@Z 1000371e f   Qt5Core:Qt5Core.dll
 0001:00002724       ??1QFile@@UAE@XZ           10003724 f   Qt5Core:Qt5Core.dll
 0001:0000272a       ?open@QFile@@UAE_NV?$QFlags@W4OpenModeFlag@QIODevice@@@@@Z 1000372a f   Qt5Core:Qt5Core.dll
 0001:00002730       ?childEvent@QObject@@MAEXPAVQChildEvent@@@Z 10003730 f   Qt5Core:Qt5Core.dll
 0001:00002736       ?connectNotify@QObject@@MAEXABVQMetaMethod@@@Z 10003736 f   Qt5Core:Qt5Core.dll
 0001:0000273c       ?customEvent@QObject@@MAEXPAVQEvent@@@Z 1000373c f   Qt5Core:Qt5Core.dll
 0001:00002742       ?disconnectNotify@QObject@@MAEXABVQMetaMethod@@@Z 10003742 f   Qt5Core:Qt5Core.dll
 0001:00002748       ?event@QObject@@UAE_NPAVQEvent@@@Z 10003748 f   Qt5Core:Qt5Core.dll
 0001:0000274e       ?eventFilter@QObject@@UAE_NPAV1@PAVQEvent@@@Z 1000374e f   Qt5Core:Qt5Core.dll
 0001:00002754       ?timerEvent@QObject@@MAEXPAVQTimerEvent@@@Z 10003754 f   Qt5Core:Qt5Core.dll
 0001:0000275a       ?dynamicMetaObject@QObjectData@@QBEPAUQMetaObject@@XZ 1000375a f   Qt5Core:Qt5Core.dll
 0001:00002760       ?qt_metacast@QObject@@UAEPAXPBD@Z 10003760 f   Qt5Core:Qt5Core.dll
 0001:00002766       ?qt_metacall@QObject@@UAEHW4Call@QMetaObject@@HPAPAX@Z 10003766 f   Qt5Core:Qt5Core.dll
 0001:0000276c       ?qRegisterResourceData@@YA_NHPBE00@Z 1000376c f   Qt5Core:Qt5Core.dll
 0001:00002772       ?qUnregisterResourceData@@YA_NHPBE00@Z 10003772 f   Qt5Core:Qt5Core.dll
 0001:00002778       ?_Xbad_alloc@std@@YAXXZ    10003778 f   msvcprt:MSVCP120.dll
 0001:0000277e       ?_Xlength_error@std@@YAXPBD@Z 1000377e f   msvcprt:MSVCP120.dll
 0001:00002784       ?_Xout_of_range@std@@YAXPBD@Z 10003784 f   msvcprt:MSVCP120.dll
 0001:0000278a       ?_Syserror_map@std@@YAPBDH@Z 1000378a f   msvcprt:MSVCP120.dll
 0001:00002790       ?_Winerror_map@std@@YAPBDH@Z 10003790 f   msvcprt:MSVCP120.dll
 0001:00002796       __purecall                 10003796 f   MSVCRT:MSVCR120.dll
 0001:0000279c       ??2@YAPAXI@Z               1000379c f   MSVCRT:MSVCR120.dll
 0001:000027a2       ??3@YAXPAX@Z               100037a2 f   MSVCRT:MSVCR120.dll
 0001:000027a8       ___atonexitinit            100037a8 f   MSVCRT:atonexit.obj
 0001:000027e4       __onexit                   100037e4 f   MSVCRT:atonexit.obj
 0001:0000288d       _atexit                    1000388d f   MSVCRT:atonexit.obj
 0001:000028a2       _memmove                   100038a2 f   MSVCRT:MSVCR120.dll
 0001:000028a8       __hypot                    100038a8 f   MSVCRT:MSVCR120.dll
 0001:000028ae       @__security_check_cookie@4 100038ae f   MSVCRT:secchk.obj
 0001:000028be       __CxxThrowException@8      100038be f   MSVCRT:MSVCR120.dll
 0001:000028c4       ___CxxFrameHandler3        100038c4 f   MSVCRT:MSVCR120.dll
 0001:000028ca       _memcpy                    100038ca f   MSVCRT:MSVCR120.dll
 0001:000028d0       ??0type_info@@AAE@ABV0@@Z  100038d0 f   MSVCRT:ti_inst.obj
 0001:000028db       ??4type_info@@AAEAAV0@ABV0@@Z 100038db f   MSVCRT:ti_inst.obj
 0001:000028e0       ??_Etype_info@@UAEPAXI@Z   100038e0 f i MSVCRT:ti_inst.obj
 0001:0000297c       _NtCurrentTeb              1000397c f i MSVCRT:crtdll.obj
 0001:00002983       __CRT_INIT@12              10003983 f   MSVCRT:crtdll.obj
 0001:00002b7a       __DllMainCRTStartup@12     10003b7a f   MSVCRT:crtdll.obj
 0001:00002cd0       __lock                     10003cd0 f   MSVCRT:MSVCR120.dll
 0001:00002cd6       __unlock                   10003cd6 f   MSVCRT:MSVCR120.dll
 0001:00002cdc       __calloc_crt               10003cdc f   MSVCRT:MSVCR120.dll
 0001:00002ce2       ___dllonexit               10003ce2 f   MSVCRT:MSVCR120.dll
 0001:00002cf0       __SEH_prolog4              10003cf0 f   MSVCRT:sehprolg4.obj
 0001:00002d35       __SEH_epilog4              10003d35 f   MSVCRT:sehprolg4.obj
 0001:00002d49       __except_handler4          10003d49 f   MSVCRT:chandler4gs.obj
 0001:00002d6c       ___raise_securityfailure   10003d6c f   MSVCRT:gs_report.obj
 0001:00002da9       ___report_gsfailure        10003da9 f   MSVCRT:gs_report.obj
 0001:00002ea4       ___report_rangecheckfailure 10003ea4 f   MSVCRT:gs_report.obj
 0001:00002eb0       ___report_securityfailure  10003eb0 f   MSVCRT:gs_report.obj
 0001:00002f80       ___report_securityfailureEx 10003f80 f   MSVCRT:gs_report.obj
 0001:00003096       ??_M@YGXPAXIHP6EX0@Z@Z     10004096 f   MSVCRT:ehvecdtr.obj
 0001:0000311e       ?__ArrayUnwind@@YGXPAXIHP6EX0@Z@Z 1000411e f   MSVCRT:ehvecdtr.obj
 0001:0000317c       ??1type_info@@UAE@XZ       1000417c f   MSVCRT:MSVCR120.dll
 0001:00003182       ___CppXcptFilter           10004182 f   MSVCRT:MSVCR120.dll
 0001:00003188       __amsg_exit                10004188 f   MSVCRT:MSVCR120.dll
 0001:00003190       __FindPESection            10004190 f   MSVCRT:pesect.obj
 0001:000031e0       __IsNonwritableInCurrentImage 100041e0 f   MSVCRT:pesect.obj
 0001:000032a0       __ValidateImageBase        100042a0 f   MSVCRT:pesect.obj
 0001:000032d2       _free                      100042d2 f   MSVCRT:MSVCR120.dll
 0001:000032d8       ___security_init_cookie    100042d8 f   MSVCRT:gs_support.obj
 0001:00003374       _DllMain@12                10004374 f   MSVCRT:dllmain.obj
 0001:00003396       __malloc_crt               10004396 f   MSVCRT:MSVCR120.dll
 0001:0000339c       __RTC_Initialize           1000439c f   MSVCRT:initsect.obj
 0001:000033bc       __RTC_Terminate            100043bc f   MSVCRT:initsect.obj
 0001:000033dc       __initterm                 100043dc f   MSVCRT:MSVCR120.dll
 0001:000033e2       __initterm_e               100043e2 f   MSVCRT:MSVCR120.dll
 0001:000033e8       ___clean_type_info_names   100043e8 f   MSVCRT:tncleanup.obj
 0001:000033f4       __except_handler4_common   100043f4 f   MSVCRT:MSVCR120.dll
 0001:000033fa       __crt_debugger_hook        100043fa f   MSVCRT:MSVCR120.dll
 0001:00003400       ___crtUnhandledException   10004400 f   MSVCRT:MSVCR120.dll
 0001:00003406       ___crtTerminateProcess     10004406 f   MSVCRT:MSVCR120.dll
 0001:0000340c       ?terminate@@YAXXZ          1000440c f   MSVCRT:MSVCR120.dll
 0001:00003412       ___clean_type_info_names_internal 10004412 f   MSVCRT:MSVCR120.dll
 0001:00003418       _EncodePointer@4           10004418 f   kernel32:KERNEL32.dll
 0001:0000341e       _DecodePointer@4           1000441e f   kernel32:KERNEL32.dll
 0001:00003424       _IsDebuggerPresent@0       10004424 f   kernel32:KERNEL32.dll
 0001:0000342a       _IsProcessorFeaturePresent@4 1000442a f   kernel32:KERNEL32.dll
 0001:00003430       _QueryPerformanceCounter@4 10004430 f   kernel32:KERNEL32.dll
 0001:00003436       _GetCurrentProcessId@0     10004436 f   kernel32:KERNEL32.dll
 0001:0000343c       _GetCurrentThreadId@0      1000443c f   kernel32:KERNEL32.dll
 0001:00003442       _GetSystemTimeAsFileTime@4 10004442 f   kernel32:KERNEL32.dll
 0001:00003448       _DisableThreadLibraryCalls@4 10004448 f   kernel32:KERNEL32.dll
 0002:00000000       __imp__DisableThreadLibraryCalls@4 10005000     kernel32:KERNEL32.dll
 0002:00000004       __imp__GetSystemTimeAsFileTime@4 10005004     kernel32:KERNEL32.dll
 0002:00000008       __imp__GetCurrentThreadId@0 10005008     kernel32:KERNEL32.dll
 0002:0000000c       __imp__GetCurrentProcessId@0 1000500c     kernel32:KERNEL32.dll
 0002:00000010       __imp__QueryPerformanceCounter@4 10005010     kernel32:KERNEL32.dll
 0002:00000014       __imp__IsProcessorFeaturePresent@4 10005014     kernel32:KERNEL32.dll
 0002:00000018       __imp__IsDebuggerPresent@0 10005018     kernel32:KERNEL32.dll
 0002:0000001c       __imp__DecodePointer@4     1000501c     kernel32:KERNEL32.dll
 0002:00000020       __imp__EncodePointer@4     10005020     kernel32:KERNEL32.dll
 0002:00000024       \177KERNEL32_NULL_THUNK_DATA 10005024     kernel32:KERNEL32.dll
 0002:00000028       __imp_?_Xbad_alloc@std@@YAXXZ 10005028     msvcprt:MSVCP120.dll
 0002:0000002c       __imp_?_Xlength_error@std@@YAXPBD@Z 1000502c     msvcprt:MSVCP120.dll
 0002:00000030       __imp_?_Xout_of_range@std@@YAXPBD@Z 10005030     msvcprt:MSVCP120.dll
 0002:00000034       __imp_?_Syserror_map@std@@YAPBDH@Z 10005034     msvcprt:MSVCP120.dll
 0002:00000038       __imp_?_Winerror_map@std@@YAPBDH@Z 10005038     msvcprt:MSVCP120.dll
 0002:0000003c       \177MSVCP120_NULL_THUNK_DATA 1000503c     msvcprt:MSVCP120.dll
 0002:00000040       __imp___initterm_e         10005040     MSVCRT:MSVCR120.dll
 0002:00000044       __imp___initterm           10005044     MSVCRT:MSVCR120.dll
 0002:00000048       __imp___malloc_crt         10005048     MSVCRT:MSVCR120.dll
 0002:0000004c       __imp__free                1000504c     MSVCRT:MSVCR120.dll
 0002:00000050       __imp___amsg_exit          10005050     MSVCRT:MSVCR120.dll
 0002:00000054       __imp____CppXcptFilter     10005054     MSVCRT:MSVCR120.dll
 0002:00000058       __imp_??1type_info@@UAE@XZ 10005058     MSVCRT:MSVCR120.dll
 0002:0000005c       __imp___onexit             1000505c     MSVCRT:MSVCR120.dll
 0002:00000060       __imp____dllonexit         10005060     MSVCRT:MSVCR120.dll
 0002:00000064       __imp___calloc_crt         10005064     MSVCRT:MSVCR120.dll
 0002:00000068       __imp___unlock             10005068     MSVCRT:MSVCR120.dll
 0002:0000006c       __imp___lock               1000506c     MSVCRT:MSVCR120.dll
 0002:00000070       __imp__memcpy              10005070     MSVCRT:MSVCR120.dll
 0002:00000074       __imp____CxxFrameHandler3  10005074     MSVCRT:MSVCR120.dll
 0002:00000078       __imp___CxxThrowException@8 10005078     MSVCRT:MSVCR120.dll
 0002:0000007c       __imp___hypot              1000507c     MSVCRT:MSVCR120.dll
 0002:00000080       __imp__memmove             10005080     MSVCRT:MSVCR120.dll
 0002:00000084       __imp_??3@YAXPAX@Z         10005084     MSVCRT:MSVCR120.dll
 0002:00000088       __imp_??2@YAPAXI@Z         10005088     MSVCRT:MSVCR120.dll
 0002:0000008c       __imp___purecall           1000508c     MSVCRT:MSVCR120.dll
 0002:00000090       __imp___except_handler4_common 10005090     MSVCRT:MSVCR120.dll
 0002:00000094       __imp___crt_debugger_hook  10005094     MSVCRT:MSVCR120.dll
 0002:00000098       __imp____crtUnhandledException 10005098     MSVCRT:MSVCR120.dll
 0002:0000009c       __imp____crtTerminateProcess 1000509c     MSVCRT:MSVCR120.dll
 0002:000000a0       __imp____clean_type_info_names_internal 100050a0     MSVCRT:MSVCR120.dll
 0002:000000a4       __imp_?terminate@@YAXXZ    100050a4     MSVCRT:MSVCR120.dll
 0002:000000a8       \177MSVCR120_NULL_THUNK_DATA 100050a8     MSVCRT:MSVCR120.dll
 0002:000000ac       __imp_??0QChar@@QAE@UQLatin1Char@@@Z 100050ac     Qt5Core:Qt5Core.dll
 0002:000000b0       __imp_??0QByteArray@@QAE@XZ 100050b0     Qt5Core:Qt5Core.dll
 0002:000000b4       __imp_??0QByteArray@@QAE@PBDH@Z 100050b4     Qt5Core:Qt5Core.dll
 0002:000000b8       __imp_??1Connection@QMetaObject@@QAE@XZ 100050b8     Qt5Core:Qt5Core.dll
 0002:000000bc       __imp_??1QByteArray@@QAE@XZ 100050bc     Qt5Core:Qt5Core.dll
 0002:000000c0       __imp_?append@QByteArray@@QAEAAV1@PBD@Z 100050c0     Qt5Core:Qt5Core.dll
 0002:000000c4       __imp_?append@QByteArray@@QAEAAV1@ABV1@@Z 100050c4     Qt5Core:Qt5Core.dll
 0002:000000c8       __imp_??0QString@@QAE@XZ   100050c8     Qt5Core:Qt5Core.dll
 0002:000000cc       __imp_??0QString@@QAE@ABV0@@Z 100050cc     Qt5Core:Qt5Core.dll
 0002:000000d0       __imp_??1QString@@QAE@XZ   100050d0     Qt5Core:Qt5Core.dll
 0002:000000d4       __imp_??4QString@@QAEAAV0@$$QAV0@@Z 100050d4     Qt5Core:Qt5Core.dll
 0002:000000d8       __imp_?tr@QMetaObject@@QBE?AVQString@@PBD0H@Z 100050d8     Qt5Core:Qt5Core.dll
 0002:000000dc       __imp_??0QString@@QAE@ABVQByteArray@@@Z 100050dc     Qt5Core:Qt5Core.dll
 0002:000000e0       __imp_?isNull@QString@@QBE_NXZ 100050e0     Qt5Core:Qt5Core.dll
 0002:000000e4       __imp_?fromAscii_helper@QString@@CAPAU?$QTypedArrayData@G@@PBDH@Z 100050e4     Qt5Core:Qt5Core.dll
 0002:000000e8       __imp_?tr@QObject@@SA?AVQString@@PBD0H@Z 100050e8     Qt5Core:Qt5Core.dll
 0002:000000ec       __imp_??0QObject@@QAE@PAV0@@Z 100050ec     Qt5Core:Qt5Core.dll
 0002:000000f0       __imp_??1QObject@@UAE@XZ   100050f0     Qt5Core:Qt5Core.dll
 0002:000000f4       __imp_?connect@QObject@@QBE?AVConnection@QMetaObject@@PBV1@PBD1W4ConnectionType@Qt@@@Z 100050f4     Qt5Core:Qt5Core.dll
 0002:000000f8       __imp_?disconnect@QObject@@SA_NPBV1@PBD01@Z 100050f8     Qt5Core:Qt5Core.dll
 0002:000000fc       __imp_??0QEventLoop@@QAE@PAVQObject@@@Z 100050fc     Qt5Core:Qt5Core.dll
 0002:00000100       __imp_??1QEventLoop@@UAE@XZ 10005100     Qt5Core:Qt5Core.dll
 0002:00000104       __imp_?exec@QEventLoop@@QAEHV?$QFlags@W4ProcessEventsFlag@QEventLoop@@@@@Z 10005104     Qt5Core:Qt5Core.dll
 0002:00000108       __imp_?exit@QEventLoop@@QAEXH@Z 10005108     Qt5Core:Qt5Core.dll
 0002:0000010c       __imp_?readAll@QIODevice@@QAE?AVQByteArray@@XZ 1000510c     Qt5Core:Qt5Core.dll
 0002:00000110       __imp_?errorString@QIODevice@@QBE?AVQString@@XZ 10005110     Qt5Core:Qt5Core.dll
 0002:00000114       __imp_??0QUrl@@QAE@ABVQString@@W4ParsingMode@0@@Z 10005114     Qt5Core:Qt5Core.dll
 0002:00000118       __imp_??1QUrl@@QAE@XZ      10005118     Qt5Core:Qt5Core.dll
 0002:0000011c       __imp_??0QTextStream@@QAE@PAVQIODevice@@@Z 1000511c     Qt5Core:Qt5Core.dll
 0002:00000120       __imp_??1QTextStream@@UAE@XZ 10005120     Qt5Core:Qt5Core.dll
 0002:00000124       __imp_?readAll@QTextStream@@QAE?AVQString@@XZ 10005124     Qt5Core:Qt5Core.dll
 0002:00000128       __imp_??0QFile@@QAE@ABVQString@@@Z 10005128     Qt5Core:Qt5Core.dll
 0002:0000012c       __imp_??1QFile@@UAE@XZ     1000512c     Qt5Core:Qt5Core.dll
 0002:00000130       __imp_?open@QFile@@UAE_NV?$QFlags@W4OpenModeFlag@QIODevice@@@@@Z 10005130     Qt5Core:Qt5Core.dll
 0002:00000134       __imp_?childEvent@QObject@@MAEXPAVQChildEvent@@@Z 10005134     Qt5Core:Qt5Core.dll
 0002:00000138       __imp_?connectNotify@QObject@@MAEXABVQMetaMethod@@@Z 10005138     Qt5Core:Qt5Core.dll
 0002:0000013c       __imp_?customEvent@QObject@@MAEXPAVQEvent@@@Z 1000513c     Qt5Core:Qt5Core.dll
 0002:00000140       __imp_?disconnectNotify@QObject@@MAEXABVQMetaMethod@@@Z 10005140     Qt5Core:Qt5Core.dll
 0002:00000144       __imp_?event@QObject@@UAE_NPAVQEvent@@@Z 10005144     Qt5Core:Qt5Core.dll
 0002:00000148       __imp_?eventFilter@QObject@@UAE_NPAV1@PAVQEvent@@@Z 10005148     Qt5Core:Qt5Core.dll
 0002:0000014c       __imp_?timerEvent@QObject@@MAEXPAVQTimerEvent@@@Z 1000514c     Qt5Core:Qt5Core.dll
 0002:00000150       __imp_?dynamicMetaObject@QObjectData@@QBEPAUQMetaObject@@XZ 10005150     Qt5Core:Qt5Core.dll
 0002:00000154       __imp_?qt_metacast@QObject@@UAEPAXPBD@Z 10005154     Qt5Core:Qt5Core.dll
 0002:00000158       __imp_?qt_metacall@QObject@@UAEHW4Call@QMetaObject@@HPAPAX@Z 10005158     Qt5Core:Qt5Core.dll
 0002:0000015c       __imp_?staticMetaObject@QObject@@2UQMetaObject@@B 1000515c     Qt5Core:Qt5Core.dll
 0002:00000160       __imp_?qRegisterResourceData@@YA_NHPBE00@Z 10005160     Qt5Core:Qt5Core.dll
 0002:00000164       __imp_?qUnregisterResourceData@@YA_NHPBE00@Z 10005164     Qt5Core:Qt5Core.dll
 0002:00000168       __imp_?arg@QString@@QBE?AV1@ABV1@HVQChar@@@Z 10005168     Qt5Core:Qt5Core.dll
 0002:0000016c       __imp_??0QByteArray@@QAE@ABV0@@Z 1000516c     Qt5Core:Qt5Core.dll
 0002:00000170       \177Qt5Core_NULL_THUNK_DATA 10005170     Qt5Core:Qt5Core.dll
 0002:00000174       __imp_?setPassword@QAuthenticator@@QAEXABVQString@@@Z 10005174     Qt5Network:Qt5Network.dll
 0002:00000178       __imp_?setUser@QAuthenticator@@QAEXABVQString@@@Z 10005178     Qt5Network:Qt5Network.dll
 0002:0000017c       __imp_?password@QNetworkProxy@@QBE?AVQString@@XZ 1000517c     Qt5Network:Qt5Network.dll
 0002:00000180       __imp_?user@QNetworkProxy@@QBE?AVQString@@XZ 10005180     Qt5Network:Qt5Network.dll
 0002:00000184       __imp_??1QNetworkProxy@@QAE@XZ 10005184     Qt5Network:Qt5Network.dll
 0002:00000188       __imp_?error@QNetworkReply@@QBE?AW4NetworkError@1@XZ 10005188     Qt5Network:Qt5Network.dll
 0002:0000018c       __imp_?get@QNetworkAccessManager@@QAEPAVQNetworkReply@@ABVQNetworkRequest@@@Z 1000518c     Qt5Network:Qt5Network.dll
 0002:00000190       __imp_?setProxy@QNetworkAccessManager@@QAEXABVQNetworkProxy@@@Z 10005190     Qt5Network:Qt5Network.dll
 0002:00000194       __imp_??1QNetworkAccessManager@@UAE@XZ 10005194     Qt5Network:Qt5Network.dll
 0002:00000198       __imp_??0QNetworkAccessManager@@QAE@PAVQObject@@@Z 10005198     Qt5Network:Qt5Network.dll
 0002:0000019c       __imp_??1QNetworkRequest@@QAE@XZ 1000519c     Qt5Network:Qt5Network.dll
 0002:000001a0       __imp_??0QNetworkRequest@@QAE@ABVQUrl@@@Z 100051a0     Qt5Network:Qt5Network.dll
 0002:000001a4       \177Qt5Network_NULL_THUNK_DATA 100051a4     Qt5Network:Qt5Network.dll
 0002:000001a8       __imp_?newObject@QScriptEngine@@QAE?AVQScriptValue@@XZ 100051a8     Qt5Script:Qt5Script.dll
 0002:000001ac       __imp_?newFunction@QScriptEngine@@QAE?AVQScriptValue@@P6A?AV2@PAVQScriptContext@@PAV1@@ZH@Z 100051ac     Qt5Script:Qt5Script.dll
 0002:000001b0       __imp_?evaluate@QScriptEngine@@QAE?AVQScriptValue@@ABVQString@@0H@Z 100051b0     Qt5Script:Qt5Script.dll
 0002:000001b4       __imp_?globalObject@QScriptEngine@@QBE?AVQScriptValue@@XZ 100051b4     Qt5Script:Qt5Script.dll
 0002:000001b8       __imp_?throwError@QScriptContext@@QAE?AVQScriptValue@@ABVQString@@@Z 100051b8     Qt5Script:Qt5Script.dll
 0002:000001bc       __imp_?argument@QScriptContext@@QBE?AVQScriptValue@@H@Z 100051bc     Qt5Script:Qt5Script.dll
 0002:000001c0       __imp_?argumentCount@QScriptContext@@QBEHXZ 100051c0     Qt5Script:Qt5Script.dll
 0002:000001c4       __imp_?setProperty@QScriptValue@@QAEXABVQString@@ABV1@ABV?$QFlags@W4PropertyFlag@QScriptValue@@@@@Z 100051c4     Qt5Script:Qt5Script.dll
 0002:000001c8       __imp_?toString@QScriptValue@@QBE?AVQString@@XZ 100051c8     Qt5Script:Qt5Script.dll
 0002:000001cc       __imp_?isObject@QScriptValue@@QBE_NXZ 100051cc     Qt5Script:Qt5Script.dll
 0002:000001d0       __imp_??0QScriptValue@@QAE@ABV0@@Z 100051d0     Qt5Script:Qt5Script.dll
 0002:000001d4       __imp_??1QScriptValue@@QAE@XZ 100051d4     Qt5Script:Qt5Script.dll
 0002:000001d8       \177Qt5Script_NULL_THUNK_DATA 100051d8     Qt5Script:Qt5Script.dll
 0002:000001dc       __imp_?getWorkflowScriptRegistry@AppContext@U2@@SAPAVWorkflowScriptRegistry@2@XZ 100051dc     U2Core:U2Core.dll
 0002:000001e0       __imp_??0Logger@U2@@QAE@ABVQString@@@Z 100051e0     U2Core:U2Core.dll
 0002:000001e4       __imp_??1Logger@U2@@UAE@XZ 100051e4     U2Core:U2Core.dll
 0002:000001e8       __imp_?staticMetaObject@Plugin@U2@@2UQMetaObject@@B 100051e8     U2Core:U2Core.dll
 0002:000001ec       __imp_?qt_metacall@Plugin@U2@@UAEHW4Call@QMetaObject@@HPAPAX@Z 100051ec     U2Core:U2Core.dll
 0002:000001f0       __imp_?qt_metacast@Plugin@U2@@UAEPAXPBD@Z 100051f0     U2Core:U2Core.dll
 0002:000001f4       __imp_?getAppSettings@AppContext@U2@@SAPAVAppSettings@2@XZ 100051f4     U2Core:U2Core.dll
 0002:000001f8       __imp_??1Plugin@U2@@UAE@XZ 100051f8     U2Core:U2Core.dll
 0002:000001fc       __imp_??0Plugin@U2@@QAE@ABVQString@@0_NW4PluginState@1@@Z 100051fc     U2Core:U2Core.dll
 0002:00000200       __imp_?getProxyByUrl@NetworkConfiguration@U2@@QBE?AVQNetworkProxy@@ABVQUrl@@@Z 10005200     U2Core:U2Core.dll
 0002:00000204       __imp_?trace@Logger@U2@@QAEXABVQString@@@Z 10005204     U2Core:U2Core.dll
 0002:00000208       \177U2Core_NULL_THUNK_DATA 10005208     U2Core:U2Core.dll
 0002:0000020c       __imp_?registerScriptFactory@WorkflowScriptRegistry@U2@@QAEXPAVWorkflowScriptFactory@2@@Z 1000520c     U2Lang:U2Lang.dll
 0002:00000210       __imp_??1WorkflowScriptFactory@U2@@UAE@XZ 10005210     U2Lang:U2Lang.dll
 0002:00000214       \177U2Lang_NULL_THUNK_DATA 10005214     U2Lang:U2Lang.dll
 0002:00000218       ___xc_a                    10005218     MSVCRT:cinitexe.obj
 0002:00000264       ___xc_z                    10005264     MSVCRT:cinitexe.obj
 0002:00000268       ___xi_a                    10005268     MSVCRT:cinitexe.obj
 0002:00000274       ___xi_z                    10005274     MSVCRT:cinitexe.obj
 0002:000002b8       ??_C@_00CNPNBAHC@?$AA@     100052b8     LinkDataScriptLibrary.obj
 0002:000002c0       ??_7error_category@std@@6B@ 100052c0     LinkDataScriptLibrary.obj
 0002:000002dc       ??_7_Generic_error_category@std@@6B@ 100052dc     LinkDataScriptLibrary.obj
 0002:000002f4       ??_C@_07DCLBNMLN@generic?$AA@ 100052f4     LinkDataScriptLibrary.obj
 0002:000002fc       ??_C@_0O@BFJCFAAK@unknown?5error?$AA@ 100052fc     LinkDataScriptLibrary.obj
 0002:00000310       ??_7_Iostream_error_category@std@@6B@ 10005310     LinkDataScriptLibrary.obj
 0002:00000328       ??_C@_08LLGCOLLL@iostream?$AA@ 10005328     LinkDataScriptLibrary.obj
 0002:00000334       ??_C@_0BG@PADBLCHM@iostream?5stream?5error?$AA@ 10005334     LinkDataScriptLibrary.obj
 0002:00000350       ??_7_System_error_category@std@@6B@ 10005350     LinkDataScriptLibrary.obj
 0002:00000368       ??_C@_06FHFOAHML@system?$AA@ 10005368     LinkDataScriptLibrary.obj
 0002:00000370       ??_C@_0L@JLHNEGIN@Algorithms?$AA@ 10005370     LinkDataScriptLibrary.obj
 0002:0000037c       ??_C@_07PGLPGHFC@Console?$AA@ 1000537c     LinkDataScriptLibrary.obj
 0002:00000384       ??_C@_0O@BOFHOPCF@Core?5Services?$AA@ 10005384     LinkDataScriptLibrary.obj
 0002:00000394       ??_C@_0N@PPADAKBM@Input?1Output?$AA@ 10005394     LinkDataScriptLibrary.obj
 0002:000003a4       ??_C@_0M@KPPBKPKK@Performance?$AA@ 100053a4     LinkDataScriptLibrary.obj
 0002:000003b0       ??_C@_07BFDHHBBI@Scripts?$AA@ 100053b0     LinkDataScriptLibrary.obj
 0002:000003b8       ??_C@_05EEGKELMG@Tasks?$AA@ 100053b8     LinkDataScriptLibrary.obj
 0002:000003c0       ??_C@_0P@NIIOBHGA@User?5Interface?$AA@ 100053c0     LinkDataScriptLibrary.obj
 0002:000003d0       ??_C@_0N@JINCGGMN@User?5Actions?$AA@ 100053d0     LinkDataScriptLibrary.obj
 0002:000003e4       ??_7LinkDataRequestHandler@U2@@6B@ 100053e4     LinkDataScriptLibrary.obj
 0002:00000410       ??_C@_0CJ@FKLHOJPJ@http?3?1?1linkdata?4org?1api?11?1?$CF1?1?$CF2_@ 10005410     LinkDataScriptLibrary.obj
 0002:0000043c       ??_C@_08FGLJJMHG@LinkData?$AA@ 1000543c     LinkDataScriptLibrary.obj
 0002:00000448       ??_C@_08NOEPOPLB@userdata?$AA@ 10005448     LinkDataScriptLibrary.obj
 0002:00000458       ??_C@_0EG@MIMJHOBC@1onProxyAuthenticationRequired?$CIc@ 10005458     LinkDataScriptLibrary.obj
 0002:000004a0       ??_C@_09GIEBNLLG@fetchFile?$AA@ 100054a0     LinkDataScriptLibrary.obj
 0002:000004ac       ??_C@_0CD@POCKECPA@?3?1linkdata_support?1src?1linkdata?4@ 100054ac     LinkDataScriptLibrary.obj
 0002:000004d0       ??_C@_0BL@BGNMMMDF@LinkData?5script?5registered?$AA@ 100054d0     LinkDataScriptLibrary.obj
 0002:000004ec       ??_C@_0BO@BLHIPPFC@Incorrect?5number?5of?5arguments?$AA@ 100054ec     LinkDataScriptLibrary.obj
 0002:0000050c       ??_C@_0BB@HMGGCEBG@Invalid?5argument?$AA@ 1000550c     LinkDataScriptLibrary.obj
 0002:00000520       ??_C@_0CE@MLPLGPCI@1sl_onReplyFinished?$CIQNetworkRepl@ 10005520     LinkDataScriptLibrary.obj
 0002:00000544       ??_C@_0BK@GPCAEHPO@2finished?$CIQNetworkReply?$CK?$CJ?$AA@ 10005544     LinkDataScriptLibrary.obj
 0002:00000560       ??_C@_0EE@HJDHBBIC@2proxyAuthenticationRequired?$CIcon@ 10005560     LinkDataScriptLibrary.obj
 0002:000005a4       ??_C@_01PKGAHCOL@?$CJ?$AA@ 100055a4     LinkDataScriptLibrary.obj
 0002:000005a8       ??_C@_01ODHLEDKK@?$CI?$AA@ 100055a8     LinkDataScriptLibrary.obj
 0002:000005ac       ??_C@_0BB@LGOPIMKM@Invalid?5response?$AA@ 100055ac     LinkDataScriptLibrary.obj
 0002:000005c0       ??_C@_0BA@JFNIOLAK@string?5too?5long?$AA@ 100055c0     LinkDataScriptLibrary.obj
 0002:000005d0       ??_C@_0BI@CFPLBAOH@invalid?5string?5position?$AA@ 100055d0     LinkDataScriptLibrary.obj
 0002:000005ec       ??_7LinkDataSupportPlugin@U2@@6B@ 100055ec     LinkDataSupportPlugin.obj
 0002:0000061c       ??_7LinkDataScriptFactory@U2@@6B@ 1000561c     LinkDataSupportPlugin.obj
 0002:00000624       ??_C@_0BB@KCFKHPBE@LinkData?5Support?$AA@ 10005624     LinkDataSupportPlugin.obj
 0002:000010d4       ?value@?$integral_constant@_N$0A@@std@@2_NB 100060d4     MSVCRT:ti_inst.obj
 0002:000010d5       ?value@?$integral_constant@_N$00@std@@2_NB 100060d5     MSVCRT:ti_inst.obj
 0002:000010dc       ??_7type_info@@6B@         100060dc     MSVCRT:ti_inst.obj
 0002:000010e0       __pRawDllMain              100060e0     MSVCRT:crtdll.obj
 0002:000010e0       __pDefaultRawDllMain       100060e0     MSVCRT:crtdll.obj
 0002:000010ec       ?ProcessDetach@NativeDll@<CrtImplementationDetails>@@0IB 100060ec     MSVCRT:initsect.obj
 0002:000010f0       ?ProcessAttach@NativeDll@<CrtImplementationDetails>@@0IB 100060f0     MSVCRT:initsect.obj
 0002:000010f4       ?ThreadAttach@NativeDll@<CrtImplementationDetails>@@0IB 100060f4     MSVCRT:initsect.obj
 0002:000010f8       ?ThreadDetach@NativeDll@<CrtImplementationDetails>@@0IB 100060f8     MSVCRT:initsect.obj
 0002:000010fc       ?ProcessVerifier@NativeDll@<CrtImplementationDetails>@@0IB 100060fc     MSVCRT:initsect.obj
 0002:00001100       __load_config_used         10006100     MSVCRT:loadcfg.obj
 0002:000011c0       ??_R4error_category@std@@6B@ 100061c0     LinkDataScriptLibrary.obj
 0002:000011d4       ??_R3error_category@std@@8 100061d4     LinkDataScriptLibrary.obj
 0002:000011e4       ??_R2error_category@std@@8 100061e4     LinkDataScriptLibrary.obj
 0002:000011ec       ??_R1A@?0A@EA@error_category@std@@8 100061ec     LinkDataScriptLibrary.obj
 0002:00001208       ??_R4_Generic_error_category@std@@6B@ 10006208     LinkDataScriptLibrary.obj
 0002:0000121c       ??_R3_Generic_error_category@std@@8 1000621c     LinkDataScriptLibrary.obj
 0002:0000122c       ??_R2_Generic_error_category@std@@8 1000622c     LinkDataScriptLibrary.obj
 0002:00001238       ??_R1A@?0A@EA@_Generic_error_category@std@@8 10006238     LinkDataScriptLibrary.obj
 0002:00001254       ??_R4_Iostream_error_category@std@@6B@ 10006254     LinkDataScriptLibrary.obj
 0002:00001268       ??_R3_Iostream_error_category@std@@8 10006268     LinkDataScriptLibrary.obj
 0002:00001278       ??_R2_Iostream_error_category@std@@8 10006278     LinkDataScriptLibrary.obj
 0002:00001288       ??_R1A@?0A@EA@_Iostream_error_category@std@@8 10006288     LinkDataScriptLibrary.obj
 0002:000012a4       ??_R4_System_error_category@std@@6B@ 100062a4     LinkDataScriptLibrary.obj
 0002:000012b8       ??_R3_System_error_category@std@@8 100062b8     LinkDataScriptLibrary.obj
 0002:000012c8       ??_R2_System_error_category@std@@8 100062c8     LinkDataScriptLibrary.obj
 0002:000012d8       ??_R1A@?0A@EA@_System_error_category@std@@8 100062d8     LinkDataScriptLibrary.obj
 0002:000012f4       ??_R1A@?0A@EA@QObject@@8   100062f4     LinkDataScriptLibrary.obj
 0002:00001310       ??_R3QObject@@8            10006310     LinkDataScriptLibrary.obj
 0002:00001320       ??_R2QObject@@8            10006320     LinkDataScriptLibrary.obj
 0002:00001328       ??_R4LinkDataRequestHandler@U2@@6B@ 10006328     LinkDataScriptLibrary.obj
 0002:0000133c       ??_R3LinkDataRequestHandler@U2@@8 1000633c     LinkDataScriptLibrary.obj
 0002:0000134c       ??_R2LinkDataRequestHandler@U2@@8 1000634c     LinkDataScriptLibrary.obj
 0002:00001358       ??_R1A@?0A@EA@LinkDataRequestHandler@U2@@8 10006358     LinkDataScriptLibrary.obj
 0002:00001374       ??_R4LinkDataSupportPlugin@U2@@6B@ 10006374     LinkDataSupportPlugin.obj
 0002:00001388       ??_R3LinkDataSupportPlugin@U2@@8 10006388     LinkDataSupportPlugin.obj
 0002:00001398       ??_R2LinkDataSupportPlugin@U2@@8 10006398     LinkDataSupportPlugin.obj
 0002:000013a8       ??_R1A@?0A@EA@LinkDataSupportPlugin@U2@@8 100063a8     LinkDataSupportPlugin.obj
 0002:000013c4       ??_R1A@?0A@EA@Plugin@U2@@8 100063c4     LinkDataSupportPlugin.obj
 0002:000013e0       ??_R3Plugin@U2@@8          100063e0     LinkDataSupportPlugin.obj
 0002:000013f0       ??_R2Plugin@U2@@8          100063f0     LinkDataSupportPlugin.obj
 0002:000013fc       ??_R4LinkDataScriptFactory@U2@@6B@ 100063fc     LinkDataSupportPlugin.obj
 0002:00001410       ??_R3LinkDataScriptFactory@U2@@8 10006410     LinkDataSupportPlugin.obj
 0002:00001420       ??_R2LinkDataScriptFactory@U2@@8 10006420     LinkDataSupportPlugin.obj
 0002:0000142c       ??_R1A@?0A@EA@LinkDataScriptFactory@U2@@8 1000642c     LinkDataSupportPlugin.obj
 0002:00001448       ??_R1A@?0A@EA@WorkflowScriptFactory@U2@@8 10006448     LinkDataSupportPlugin.obj
 0002:00001464       ??_R3WorkflowScriptFactory@U2@@8 10006464     LinkDataSupportPlugin.obj
 0002:00001474       ??_R2WorkflowScriptFactory@U2@@8 10006474     LinkDataSupportPlugin.obj
 0002:0000147c       ??_R4type_info@@6B@        1000647c     MSVCRT:ti_inst.obj
 0002:00001490       ??_R3type_info@@8          10006490     MSVCRT:ti_inst.obj
 0002:000014a0       ??_R2type_info@@8          100064a0     MSVCRT:ti_inst.obj
 0002:000014a8       ??_R1A@?0A@EA@type_info@@8 100064a8     MSVCRT:ti_inst.obj
 0002:000014d0       ___safe_se_handler_table   100064d0     <linker-defined>
 0002:00001528       ___rtc_iaa                 10006528     MSVCRT:initsect.obj
 0002:0000152c       ___rtc_izz                 1000652c     MSVCRT:initsect.obj
 0002:00001530       ___rtc_taa                 10006530     MSVCRT:initsect.obj
 0002:00001534       ___rtc_tzz                 10006534     MSVCRT:initsect.obj
 0002:00001c2c       __IMPORT_DESCRIPTOR_U2Core 10006c2c     U2Core:U2Core.dll
 0002:00001c40       __IMPORT_DESCRIPTOR_U2Lang 10006c40     U2Lang:U2Lang.dll
 0002:00001c54       __IMPORT_DESCRIPTOR_Qt5Script 10006c54     Qt5Script:Qt5Script.dll
 0002:00001c68       __IMPORT_DESCRIPTOR_Qt5Network 10006c68     Qt5Network:Qt5Network.dll
 0002:00001c7c       __IMPORT_DESCRIPTOR_Qt5Core 10006c7c     Qt5Core:Qt5Core.dll
 0002:00001c90       __IMPORT_DESCRIPTOR_MSVCP120 10006c90     msvcprt:MSVCP120.dll
 0002:00001ca4       __IMPORT_DESCRIPTOR_MSVCR120 10006ca4     MSVCRT:MSVCR120.dll
 0002:00001cb8       __IMPORT_DESCRIPTOR_KERNEL32 10006cb8     kernel32:KERNEL32.dll
 0002:00001ccc       __NULL_IMPORT_DESCRIPTOR   10006ccc     U2Core:U2Core.dll
 0003:00000000       ?_Generic_object@?$_Error_objects@H@std@@2V_Generic_error_category@2@A 10009000     LinkDataScriptLibrary.obj
 0003:00000004       ?_Iostream_object@?$_Error_objects@H@std@@2V_Iostream_error_category@2@A 10009004     LinkDataScriptLibrary.obj
 0003:00000008       ?_System_object@?$_Error_objects@H@std@@2V_System_error_category@2@A 10009008     LinkDataScriptLibrary.obj
 0003:0000000c       ?staticMetaObject@LinkDataRequestHandler@U2@@2UQMetaObject@@B 1000900c     moc_LinkDataScriptLibrary.obj
 0003:00000024       ?staticMetaObject@LinkDataSupportPlugin@U2@@2UQMetaObject@@B 10009024     moc_LinkDataSupportPlugin.obj
 0003:0000003c       ___security_cookie         1000903c     MSVCRT:gs_cookie.obj
 0003:00000040       ___security_cookie_complement 10009040     MSVCRT:gs_cookie.obj
 0003:00000050       ___native_dllmain_reason   10009050     MSVCRT:natstart.obj
 0003:00000054       ??_R0?AVerror_category@std@@@8 10009054     LinkDataScriptLibrary.obj
 0003:00000078       ??_R0?AV_Generic_error_category@std@@@8 10009078     LinkDataScriptLibrary.obj
 0003:000000a4       ??_R0?AV_Iostream_error_category@std@@@8 100090a4     LinkDataScriptLibrary.obj
 0003:000000d0       ??_R0?AV_System_error_category@std@@@8 100090d0     LinkDataScriptLibrary.obj
 0003:000000fc       ??_R0?AVQObject@@@8        100090fc     LinkDataScriptLibrary.obj
 0003:00000114       ??_R0?AVLinkDataRequestHandler@U2@@@8 10009114     LinkDataScriptLibrary.obj
 0003:0000013c       ??_R0?AVLinkDataSupportPlugin@U2@@@8 1000913c     LinkDataSupportPlugin.obj
 0003:00000164       ??_R0?AVPlugin@U2@@@8      10009164     LinkDataSupportPlugin.obj
 0003:0000017c       ??_R0?AVLinkDataScriptFactory@U2@@@8 1000917c     LinkDataSupportPlugin.obj
 0003:000001a4       ??_R0?AVWorkflowScriptFactory@U2@@@8 100091a4     LinkDataSupportPlugin.obj
 0003:000001cc       ??_R0?AVtype_info@@@8      100091cc     MSVCRT:ti_inst.obj
 0003:00000240       ?id@?$num_put@DV?$back_insert_iterator@V?$basic_string@DU?$char_traits@D@std@@V?$allocator@D@2@@std@@@std@@@std@@2V0locale@2@A 10009240     LinkDataScriptLibrary.obj
 0003:00000244       ?id@?$num_put@_WV?$back_insert_iterator@V?$basic_string@_WU?$char_traits@_W@std@@V?$allocator@_W@2@@std@@@std@@@std@@2V0locale@2@A 10009244     LinkDataScriptLibrary.obj
 0003:00000254       ?dummy@?A0x896ef0f2@@3Uinitializer@1@A 10009254     qrc_linkdata_support.obj
 0003:00000580       ?__type_info_root_node@@3U__type_info_node@@A 10009580     MSVCRT:tncleanup.obj
 0003:00000588       ___native_startup_lock     10009588     <common>
 0003:0000058c       ___native_startup_state    1000958c     <common>
 0003:00000590       ___dyn_tls_init_callback   10009590     <common>
 0003:00000594       ___onexitend               10009594     <common>
 0003:00000598       ___onexitbegin             10009598     <common>

 entry point at        0001:00002b7a

 Static symbols

 0000:ffff4000       .debug$S                   10000000     MSVCRT:MSVCR120.dll
 0000:ffff4000       .debug$S                   10000000     MSVCRT:MSVCR120.dll
 0000:ffff4000       .debug$S                   10000000     MSVCRT:MSVCR120.dll
 0000:ffff4000       .debug$S                   10000000     MSVCRT:MSVCR120.dll
 0000:ffff4000       .debug$S                   10000000     MSVCRT:MSVCR120.dll
 0000:ffff4000       .debug$S                   10000000     MSVCRT:MSVCR120.dll
 0000:ffff4000       .debug$S                   10000000     MSVCRT:MSVCR120.dll
 0000:ffff4000       .debug$S                   10000000     Qt5Core:Qt5Core.dll
 0000:ffff4000       .debug$S                   10000000     Qt5Core:Qt5Core.dll
 0000:ffff4000       .debug$S                   10000000     Qt5Core:Qt5Core.dll
 0000:ffff4000       .debug$S                   10000000     Qt5Core:Qt5Core.dll
 0000:ffff4000       .debug$S                   10000000     Qt5Core:Qt5Core.dll
 0000:ffff4000       .debug$S                   10000000     Qt5Core:Qt5Core.dll
 0000:ffff4000       .debug$S                   10000000     Qt5Core:Qt5Core.dll
 0000:ffff4000       .debug$S                   10000000     Qt5Core:Qt5Core.dll
 0000:ffff4000       .debug$S                   10000000     Qt5Core:Qt5Core.dll
 0000:ffff4000       .debug$S                   10000000     Qt5Core:Qt5Core.dll
 0000:ffff4000       .debug$S                   10000000     Qt5Core:Qt5Core.dll
 0000:ffff4000       .debug$S                   10000000     Qt5Core:Qt5Core.dll
 0000:ffff4000       .debug$S                   10000000     Qt5Core:Qt5Core.dll
 0000:ffff4000       .debug$S                   10000000     Qt5Core:Qt5Core.dll
 0000:ffff4000       .debug$S                   10000000     Qt5Core:Qt5Core.dll
 0001:fffff000       __ehhandler$?_Copy@?$basic_string@DU?$char_traits@D@std@@V?$allocator@D@2@@std@@QAEXII@Z 10000000 f   moc_LinkDataSupportPlugin.obj
 0000:ffff4000       .debug$S                   10000000     Qt5Core:Qt5Core.dll
 0000:ffff4000       .debug$S                   10000000     Qt5Core:Qt5Core.dll
 0000:ffff4000       .debug$S                   10000000     Qt5Core:Qt5Core.dll
 0000:ffff4000       .debug$S                   10000000     Qt5Core:Qt5Core.dll
 0000:ffff4000       .debug$S                   10000000     Qt5Core:Qt5Core.dll
 0000:ffff4000       .debug$S                   10000000     Qt5Core:Qt5Core.dll
 0002:ffffb000       __catchsym$?_Copy@?$basic_string@DU?$char_traits@D@std@@V?$allocator@D@2@@std@@QAEXII@Z$5 10000000     moc_LinkDataSupportPlugin.obj
 0000:ffff4000       .debug$S                   10000000     MSVCRT:MSVCR120.dll
 0000:ffff4000       .debug$S                   10000000     MSVCRT:MSVCR120.dll
 0000:ffff4000       .debug$S                   10000000     MSVCRT:MSVCR120.dll
 0000:ffff4000       .debug$S                   10000000     MSVCRT:MSVCR120.dll
 0000:ffff4000       .debug$S                   10000000     Qt5Core:Qt5Core.dll
 0002:ffffb000       ?_Generic_object$initializer$@?$_Error_objects@H@std@@2P6AXXZA 10000000     moc_LinkDataSupportPlugin.obj
 0002:ffffb000       ?_Iostream_object$initializer$@?$_Error_objects@H@std@@2P6AXXZA 10000000     moc_LinkDataSupportPlugin.obj
 0002:ffffb000       ?_System_object$initializer$@?$_Error_objects@H@std@@2P6AXXZA 10000000     moc_LinkDataSupportPlugin.obj
 0000:ffff4000       .debug$S                   10000000     Qt5Core:Qt5Core.dll
 0000:ffff4000       .debug$S                   10000000     Qt5Network:Qt5Network.dll
 0000:ffff4000       .debug$S                   10000000     Qt5Network:Qt5Network.dll
 0000:ffff4000       .debug$S                   10000000     Qt5Network:Qt5Network.dll
 0000:ffff4000       .debug$S                   10000000     Qt5Network:Qt5Network.dll
 0000:ffff4000       .debug$S                   10000000     Qt5Network:Qt5Network.dll
 0000:ffff4000       .debug$S                   10000000     Qt5Network:Qt5Network.dll
 0000:ffff4000       .debug$S                   10000000     Qt5Network:Qt5Network.dll
 0000:ffff4000       .debug$S                   10000000     Qt5Network:Qt5Network.dll
 0001:fffff000       __ehhandler$?_Copy@?$basic_string@DU?$char_traits@D@std@@V?$allocator@D@2@@std@@QAEXII@Z 10000000 f   moc_LinkDataScriptLibrary.obj
 0000:ffff4000       .debug$S                   10000000     Qt5Network:Qt5Network.dll
 0000:ffff4000       .debug$S                   10000000     Qt5Network:Qt5Network.dll
 0000:ffff4000       .debug$S                   10000000     Qt5Network:Qt5Network.dll
 0000:ffff4000       .debug$S                   10000000     Qt5Network:Qt5Network.dll
 0000:ffff4000       .debug$S                   10000000     Qt5Core:Qt5Core.dll
 0000:ffff4000       .debug$S                   10000000     Qt5Script:Qt5Script.dll
 0002:ffffb000       __catchsym$?_Copy@?$basic_string@DU?$char_traits@D@std@@V?$allocator@D@2@@std@@QAEXII@Z$5 10000000     moc_LinkDataScriptLibrary.obj
 0000:ffff4000       .debug$S                   10000000     MSVCRT:MSVCR120.dll
 0000:ffff4000       .debug$S                   10000000     MSVCRT:MSVCR120.dll
 0000:ffff4000       .debug$S                   10000000     MSVCRT:MSVCR120.dll
 0000:ffff4000       .debug$S                   10000000     MSVCRT:MSVCR120.dll
 0000:ffff4000       .debug$S                   10000000     Qt5Script:Qt5Script.dll
 0002:ffffb000       ?_Generic_object$initializer$@?$_Error_objects@H@std@@2P6AXXZA 10000000     moc_LinkDataScriptLibrary.obj
 0002:ffffb000       ?_Iostream_object$initializer$@?$_Error_objects@H@std@@2P6AXXZA 10000000     moc_LinkDataScriptLibrary.obj
 0002:ffffb000       ?_System_object$initializer$@?$_Error_objects@H@std@@2P6AXXZA 10000000     moc_LinkDataScriptLibrary.obj
 0000:ffff4000       .debug$S                   10000000     Qt5Script:Qt5Script.dll
 0000:ffff4000       .debug$S                   10000000     Qt5Script:Qt5Script.dll
 0000:ffff4000       .debug$S                   10000000     Qt5Script:Qt5Script.dll
 0000:ffff4000       .debug$S                   10000000     Qt5Script:Qt5Script.dll
 0000:ffff4000       .debug$S                   10000000     Qt5Script:Qt5Script.dll
 0000:ffff4000       .debug$S                   10000000     Qt5Script:Qt5Script.dll
 0001:fffff000       __ehhandler$?_Copy@?$basic_string@DU?$char_traits@D@std@@V?$allocator@D@2@@std@@QAEXII@Z 10000000 f   LinkDataSupportPlugin.obj
 0000:ffff4000       .debug$S                   10000000     Qt5Script:Qt5Script.dll
 0000:ffff4000       .debug$S                   10000000     Qt5Script:Qt5Script.dll
 0000:ffff4000       .debug$S                   10000000     Qt5Script:Qt5Script.dll
 0000:ffff4000       .debug$S                   10000000     Qt5Script:Qt5Script.dll
 0000:ffff4000       .debug$S                   10000000     Qt5Core:Qt5Core.dll
 0000:ffff4000       .debug$S                   10000000     U2Lang:U2Lang.dll
 0000:ffff4000       .debug$S                   10000000     U2Lang:U2Lang.dll
 0000:ffff4000       .debug$S                   10000000     Qt5Core:Qt5Core.dll
 0000:ffff4000       .debug$S                   10000000     U2Core:U2Core.dll
 0000:ffff4000       .debug$S                   10000000     U2Core:U2Core.dll
 0002:ffffb000       __catchsym$?_Copy@?$basic_string@DU?$char_traits@D@std@@V?$allocator@D@2@@std@@QAEXII@Z$5 10000000     LinkDataSupportPlugin.obj
 0000:ffff4000       .debug$S                   10000000     MSVCRT:MSVCR120.dll
 0000:ffff4000       .debug$S                   10000000     MSVCRT:MSVCR120.dll
 0000:ffff4000       .debug$S                   10000000     MSVCRT:MSVCR120.dll
 0000:ffff4000       .debug$S                   10000000     MSVCRT:MSVCR120.dll
 0000:ffff4000       .debug$S                   10000000     MSVCRT:MSVCR120.dll
 0000:ffff4000       .debug$S                   10000000     MSVCRT:MSVCR120.dll
 0002:ffffb000       ?_Generic_object$initializer$@?$_Error_objects@H@std@@2P6AXXZA 10000000     LinkDataSupportPlugin.obj
 0002:ffffb000       ?_Iostream_object$initializer$@?$_Error_objects@H@std@@2P6AXXZA 10000000     LinkDataSupportPlugin.obj
 0002:ffffb000       ?_System_object$initializer$@?$_Error_objects@H@std@@2P6AXXZA 10000000     LinkDataSupportPlugin.obj
 0000:ffff4000       .debug$S                   10000000     U2Core:U2Core.dll
 0000:ffff4000       .debug$S                   10000000     U2Core:U2Core.dll
 0000:ffff4000       .debug$S                   10000000     U2Core:U2Core.dll
 0000:ffff4000       .debug$S                   10000000     U2Core:U2Core.dll
 0000:ffff4000       .debug$S                   10000000     U2Core:U2Core.dll
 0000:ffff4000       .debug$S                   10000000     U2Core:U2Core.dll
 0000:ffff4000       .debug$S                   10000000     U2Core:U2Core.dll
 0000:ffff4000       .debug$S                   10000000     U2Core:U2Core.dll
 0000:ffff4000       .debug$S                   10000000     U2Core:U2Core.dll
 0000:ffff4000       .debug$S                   10000000     Qt5Core:Qt5Core.dll
 0000:ffff4000       .debug$S                   10000000     Qt5Core:Qt5Core.dll
 0000:ffff4000       .debug$S                   10000000     Qt5Core:Qt5Core.dll
 0000:ffff4000       .debug$S                   10000000     Qt5Core:Qt5Core.dll
 0000:ffff4000       .debug$S                   10000000     Qt5Core:Qt5Core.dll
 0000:ffff4000       .debug$S                   10000000     Qt5Core:Qt5Core.dll
 0000:ffff4000       .debug$S                   10000000     Qt5Core:Qt5Core.dll
 0000:ffff4000       .debug$S                   10000000     Qt5Core:Qt5Core.dll
 0000:ffff4000       .debug$S                   10000000     Qt5Core:Qt5Core.dll
 0000:ffff4000       .debug$S                   10000000     Qt5Core:Qt5Core.dll
 0000:ffff4000       .debug$S                   10000000     Qt5Core:Qt5Core.dll
 0000:ffff4000       .debug$S                   10000000     Qt5Core:Qt5Core.dll
 0000:ffff4000       .debug$S                   10000000     Qt5Core:Qt5Core.dll
 0000:ffff4000       .debug$S                   10000000     Qt5Core:Qt5Core.dll
 0000:ffff4000       .debug$S                   10000000     Qt5Core:Qt5Core.dll
 0000:ffff4000       .debug$S                   10000000     Qt5Core:Qt5Core.dll
 0000:ffff4000       .debug$S                   10000000     Qt5Core:Qt5Core.dll
 0000:ffff4000       .debug$S                   10000000     Qt5Core:Qt5Core.dll
 0000:ffff4000       .debug$S                   10000000     Qt5Core:Qt5Core.dll
 0000:ffff4000       .debug$S                   10000000     Qt5Core:Qt5Core.dll
 0000:ffff4000       .debug$S                   10000000     Qt5Core:Qt5Core.dll
 0000:ffff4000       .debug$S                   10000000     Qt5Core:Qt5Core.dll
 0000:ffff4000       .debug$S                   10000000     kernel32:KERNEL32.dll
 0000:ffff4000       .debug$S                   10000000     kernel32:KERNEL32.dll
 0000:ffff4000       .debug$S                   10000000     kernel32:KERNEL32.dll
 0000:ffff4000       .debug$S                   10000000     kernel32:KERNEL32.dll
 0000:ffff4000       .debug$S                   10000000     kernel32:KERNEL32.dll
 0000:ffff4000       .debug$S                   10000000     kernel32:KERNEL32.dll
 0000:ffff4000       .debug$S                   10000000     kernel32:KERNEL32.dll
 0000:ffff4000       .debug$S                   10000000     kernel32:KERNEL32.dll
 0000:ffff4000       .debug$S                   10000000     kernel32:KERNEL32.dll
 0000:ffff4000       .debug$S                   10000000     msvcprt:MSVCP120.dll
 0000:ffff4000       .debug$S                   10000000     msvcprt:MSVCP120.dll
 0000:ffff4000       .debug$S                   10000000     msvcprt:MSVCP120.dll
 0000:ffff4000       .debug$S                   10000000     msvcprt:MSVCP120.dll
 0000:ffff4000       .debug$S                   10000000     msvcprt:MSVCP120.dll
 0000:ffff4000       .debug$S                   10000000     MSVCRT:MSVCR120.dll
 0000:ffff4000       .debug$S                   10000000     MSVCRT:MSVCR120.dll
 0000:ffff4000       .debug$S                   10000000     MSVCRT:MSVCR120.dll
 0000:ffff4000       .debug$S                   10000000     MSVCRT:MSVCR120.dll
 0000:ffff4000       .debug$S                   10000000     MSVCRT:MSVCR120.dll
 0000:ffff4000       .debug$S                   10000000     Qt5Core:Qt5Core.dll
 0002:ffffb010       __catchsym$?_Copy@?$basic_string@DU?$char_traits@D@std@@V?$allocator@D@2@@std@@QAEXII@Z$4 10000010     LinkDataSupportPlugin.obj
 0002:ffffb010       __catchsym$?_Copy@?$basic_string@DU?$char_traits@D@std@@V?$allocator@D@2@@std@@QAEXII@Z$4 10000010     moc_LinkDataScriptLibrary.obj
 0002:ffffb010       __catchsym$?_Copy@?$basic_string@DU?$char_traits@D@std@@V?$allocator@D@2@@std@@QAEXII@Z$4 10000010     moc_LinkDataSupportPlugin.obj
 0002:ffffb020       __unwindtable$?_Copy@?$basic_string@DU?$char_traits@D@std@@V?$allocator@D@2@@std@@QAEXII@Z 10000020     moc_LinkDataSupportPlugin.obj
 0002:ffffb020       __unwindtable$?_Copy@?$basic_string@DU?$char_traits@D@std@@V?$allocator@D@2@@std@@QAEXII@Z 10000020     moc_LinkDataScriptLibrary.obj
 0002:ffffb020       __unwindtable$?_Copy@?$basic_string@DU?$char_traits@D@std@@V?$allocator@D@2@@std@@QAEXII@Z 10000020     LinkDataSupportPlugin.obj
 0002:ffffb040       __ehfuncinfo$?_Copy@?$basic_string@DU?$char_traits@D@std@@V?$allocator@D@2@@std@@QAEXII@Z 10000040     LinkDataSupportPlugin.obj
 0002:ffffb040       __ehfuncinfo$?_Copy@?$basic_string@DU?$char_traits@D@std@@V?$allocator@D@2@@std@@QAEXII@Z 10000040     moc_LinkDataSupportPlugin.obj
 0002:ffffb040       __ehfuncinfo$?_Copy@?$basic_string@DU?$char_traits@D@std@@V?$allocator@D@2@@std@@QAEXII@Z 10000040     moc_LinkDataScriptLibrary.obj
 0002:ffffb064       __tryblocktable$?_Copy@?$basic_string@DU?$char_traits@D@std@@V?$allocator@D@2@@std@@QAEXII@Z 10000064     moc_LinkDataSupportPlugin.obj
 0002:ffffb064       __tryblocktable$?_Copy@?$basic_string@DU?$char_traits@D@std@@V?$allocator@D@2@@std@@QAEXII@Z 10000064     moc_LinkDataScriptLibrary.obj
 0002:ffffb064       __tryblocktable$?_Copy@?$basic_string@DU?$char_traits@D@std@@V?$allocator@D@2@@std@@QAEXII@Z 10000064     LinkDataSupportPlugin.obj
 0001:fffff096       __catch$?_Copy@?$basic_string@DU?$char_traits@D@std@@V?$allocator@D@2@@std@@QAEXII@Z$0 10000096 f   moc_LinkDataScriptLibrary.obj
 0001:fffff096       __catch$?_Copy@?$basic_string@DU?$char_traits@D@std@@V?$allocator@D@2@@std@@QAEXII@Z$0 10000096 f   moc_LinkDataSupportPlugin.obj
 0001:fffff096       __catch$?_Copy@?$basic_string@DU?$char_traits@D@std@@V?$allocator@D@2@@std@@QAEXII@Z$0 10000096 f   LinkDataSupportPlugin.obj
 0001:fffff0d3       __catch$?_Copy@?$basic_string@DU?$char_traits@D@std@@V?$allocator@D@2@@std@@QAEXII@Z$1 100000d3 f   moc_LinkDataScriptLibrary.obj
 0001:fffff0d3       __catch$?_Copy@?$basic_string@DU?$char_traits@D@std@@V?$allocator@D@2@@std@@QAEXII@Z$1 100000d3 f   moc_LinkDataSupportPlugin.obj
 0001:fffff0d3       __catch$?_Copy@?$basic_string@DU?$char_traits@D@std@@V?$allocator@D@2@@std@@QAEXII@Z$1 100000d3 f   LinkDataSupportPlugin.obj
 0001:00000000       ??__E?_Generic_object@?$_Error_objects@H@std@@2V_Generic_error_category@2@A@@YAXXZ 10001000 f   LinkDataScriptLibrary.obj
 0001:00000010       ??__E?_Iostream_object@?$_Error_objects@H@std@@2V_Iostream_error_category@2@A@@YAXXZ 10001010 f   LinkDataScriptLibrary.obj
 0001:00000020       ??__E?_System_object@?$_Error_objects@H@std@@2V_System_error_category@2@A@@YAXXZ 10001020 f   LinkDataScriptLibrary.obj
 0001:00000030       ??__ELINKDATA_API_URL@U2@@YAXXZ 10001030 f   LinkDataScriptLibrary.obj
 0001:00000050       ??__ELINKDATA_OBJ_NAME@U2@@YAXXZ 10001050 f   LinkDataScriptLibrary.obj
 0001:00000070       ??__ELINKDATA_USERDATA_OBJ_NAME@U2@@YAXXZ 10001070 f   LinkDataScriptLibrary.obj
 0001:00000090       ??__EalgoLog@U2@@YAXXZ     10001090 f   LinkDataScriptLibrary.obj
 0001:00000110       ??__EcmdLog@U2@@YAXXZ      10001110 f   LinkDataScriptLibrary.obj
 0001:00000190       ??__EcoreLog@U2@@YAXXZ     10001190 f   LinkDataScriptLibrary.obj
 0001:00000210       ??__EioLog@U2@@YAXXZ       10001210 f   LinkDataScriptLibrary.obj
 0001:00000290       ??__EperfLog@U2@@YAXXZ     10001290 f   LinkDataScriptLibrary.obj
 0001:00000310       ??__EscriptLog@U2@@YAXXZ   10001310 f   LinkDataScriptLibrary.obj
 0001:00000390       ??__EtaskLog@U2@@YAXXZ     10001390 f   LinkDataScriptLibrary.obj
 0001:00000410       ??__EuiLog@U2@@YAXXZ       10001410 f   LinkDataScriptLibrary.obj
 0001:00000490       ??__EuserActLog@U2@@YAXXZ  10001490 f   LinkDataScriptLibrary.obj
 0001:00000510       ??__E?_Generic_object@?$_Error_objects@H@std@@2V_Generic_error_category@2@A@@YAXXZ 10001510 f   LinkDataSupportPlugin.obj
 0001:00000520       ??__E?_Iostream_object@?$_Error_objects@H@std@@2V_Iostream_error_category@2@A@@YAXXZ 10001520 f   LinkDataSupportPlugin.obj
 0001:00000530       ??__E?_System_object@?$_Error_objects@H@std@@2V_System_error_category@2@A@@YAXXZ 10001530 f   LinkDataSupportPlugin.obj
 0001:00000540       ??__E?_Generic_object@?$_Error_objects@H@std@@2V_Generic_error_category@2@A@@YAXXZ 10001540 f   moc_LinkDataScriptLibrary.obj
 0001:00000550       ??__E?_Iostream_object@?$_Error_objects@H@std@@2V_Iostream_error_category@2@A@@YAXXZ 10001550 f   moc_LinkDataScriptLibrary.obj
 0001:00000560       ??__E?_System_object@?$_Error_objects@H@std@@2V_System_error_category@2@A@@YAXXZ 10001560 f   moc_LinkDataScriptLibrary.obj
 0001:00000570       ??__E?staticMetaObject@LinkDataRequestHandler@U2@@2UQMetaObject@@B@@YAXXZ 10001570 f   moc_LinkDataScriptLibrary.obj
 0001:00000580       ??__E?_Generic_object@?$_Error_objects@H@std@@2V_Generic_error_category@2@A@@YAXXZ 10001580 f   moc_LinkDataSupportPlugin.obj
 0001:00000590       ??__E?_Iostream_object@?$_Error_objects@H@std@@2V_Iostream_error_category@2@A@@YAXXZ 10001590 f   moc_LinkDataSupportPlugin.obj
 0001:000005a0       ??__E?_System_object@?$_Error_objects@H@std@@2V_System_error_category@2@A@@YAXXZ 100015a0 f   moc_LinkDataSupportPlugin.obj
 0001:000005b0       ??__E?staticMetaObject@LinkDataSupportPlugin@U2@@2UQMetaObject@@B@@YAXXZ 100015b0 f   moc_LinkDataSupportPlugin.obj
 0001:000005c0       ??__Edummy@?A0x896ef0f2@@YAXXZ 100015c0 f   qrc_linkdata_support.obj
 0001:00000d26       __catch$?_Copy@?$basic_string@DU?$char_traits@D@std@@V?$allocator@D@2@@std@@QAEXII@Z$0 10001d26 f i LinkDataScriptLibrary.obj
 0001:00000d63       __catch$?_Copy@?$basic_string@DU?$char_traits@D@std@@V?$allocator@D@2@@std@@QAEXII@Z$1 10001d63 f i LinkDataScriptLibrary.obj
 0001:00001f30       ?readScript@U2@@YA?AVQString@@ABV2@@Z 10002f30 f   LinkDataScriptLibrary.obj
 0001:00002930       _pre_c_init                10003930 f   MSVCRT:crtdll.obj
 0001:00002b9d       ___DllMainCRTStartup       10003b9d f   MSVCRT:crtdll.obj
 0001:00002cf0       $$000000                   10003cf0     MSVCRT:sehprolg4.obj
 0001:00003105       ?ArrayUnwindFilter@@YAHPAU_EXCEPTION_POINTERS@@@Z 10004105 f   MSVCRT:ehvecdtr.obj
 0001:00003450       __unwindfunclet$??0LinkDataRequestHandler@U2@@QAE@PAVQEventLoop@@@Z$0 10004450 f   LinkDataScriptLibrary.obj
 0001:00003459       __unwindfunclet$??0LinkDataRequestHandler@U2@@QAE@PAVQEventLoop@@@Z$1 10004459 f   LinkDataScriptLibrary.obj
 0001:00003465       __ehhandler$??0LinkDataRequestHandler@U2@@QAE@PAVQEventLoop@@@Z 10004465 f   LinkDataScriptLibrary.obj
 0001:00003480       __unwindfunclet$??1LinkDataRequestHandler@U2@@UAE@XZ$0 10004480 f   LinkDataScriptLibrary.obj
 0001:00003489       __unwindfunclet$??1LinkDataRequestHandler@U2@@UAE@XZ$1 10004489 f   LinkDataScriptLibrary.obj
 0001:00003495       __ehhandler$??1LinkDataRequestHandler@U2@@UAE@XZ 10004495 f   LinkDataScriptLibrary.obj
 0001:000034b0       __unwindfunclet$??H@YA?BVQByteArray@@ABV0@PBD@Z$0 100044b0 f   LinkDataScriptLibrary.obj
 0001:000034b9       __unwindfunclet$??H@YA?BVQByteArray@@ABV0@PBD@Z$1 100044b9 f   LinkDataScriptLibrary.obj
 0001:000034d3       __ehhandler$??H@YA?BVQByteArray@@ABV0@PBD@Z 100044d3 f   LinkDataScriptLibrary.obj
 0001:000034f0       __unwindfunclet$??H@YA?BVQByteArray@@PBDABV0@@Z$0 100044f0 f   LinkDataScriptLibrary.obj
 0001:000034f9       __unwindfunclet$??H@YA?BVQByteArray@@PBDABV0@@Z$1 100044f9 f   LinkDataScriptLibrary.obj
 0001:00003513       __ehhandler$??H@YA?BVQByteArray@@PBDABV0@@Z 10004513 f   LinkDataScriptLibrary.obj
 0001:00003530       __unwindfunclet$??_GLinkDataRequestHandler@U2@@UAEPAXI@Z$0 10004530 f   LinkDataScriptLibrary.obj
 0001:00003539       __unwindfunclet$??_GLinkDataRequestHandler@U2@@UAEPAXI@Z$1 10004539 f   LinkDataScriptLibrary.obj
 0001:00003545       __ehhandler$??_GLinkDataRequestHandler@U2@@UAEPAXI@Z 10004545 f   LinkDataScriptLibrary.obj
 0001:00003560       __unwindfunclet$??__EalgoLog@U2@@YAXXZ$0 10004560 f   LinkDataScriptLibrary.obj
 0001:00003569       __ehhandler$??__EalgoLog@U2@@YAXXZ 10004569 f   LinkDataScriptLibrary.obj
 0001:00003590       __unwindfunclet$??__EcmdLog@U2@@YAXXZ$0 10004590 f   LinkDataScriptLibrary.obj
 0001:00003599       __ehhandler$??__EcmdLog@U2@@YAXXZ 10004599 f   LinkDataScriptLibrary.obj
 0001:000035c0       __unwindfunclet$??__EcoreLog@U2@@YAXXZ$0 100045c0 f   LinkDataScriptLibrary.obj
 0001:000035c9       __ehhandler$??__EcoreLog@U2@@YAXXZ 100045c9 f   LinkDataScriptLibrary.obj
 0001:000035f0       __unwindfunclet$??__EioLog@U2@@YAXXZ$0 100045f0 f   LinkDataScriptLibrary.obj
 0001:000035f9       __ehhandler$??__EioLog@U2@@YAXXZ 100045f9 f   LinkDataScriptLibrary.obj
 0001:00003620       __unwindfunclet$??__EperfLog@U2@@YAXXZ$0 10004620 f   LinkDataScriptLibrary.obj
 0001:00003629       __ehhandler$??__EperfLog@U2@@YAXXZ 10004629 f   LinkDataScriptLibrary.obj
 0001:00003650       __unwindfunclet$??__EscriptLog@U2@@YAXXZ$0 10004650 f   LinkDataScriptLibrary.obj
 0001:00003659       __ehhandler$??__EscriptLog@U2@@YAXXZ 10004659 f   LinkDataScriptLibrary.obj
 0001:00003680       __unwindfunclet$??__EtaskLog@U2@@YAXXZ$0 10004680 f   LinkDataScriptLibrary.obj
 0001:00003689       __ehhandler$??__EtaskLog@U2@@YAXXZ 10004689 f   LinkDataScriptLibrary.obj
 0001:000036b0       __unwindfunclet$??__EuiLog@U2@@YAXXZ$0 100046b0 f   LinkDataScriptLibrary.obj
 0001:000036b9       __ehhandler$??__EuiLog@U2@@YAXXZ 100046b9 f   LinkDataScriptLibrary.obj
 0001:000036e0       __unwindfunclet$??__EuserActLog@U2@@YAXXZ$0 100046e0 f   LinkDataScriptLibrary.obj
 0001:000036e9       __ehhandler$??__EuserActLog@U2@@YAXXZ 100046e9 f   LinkDataScriptLibrary.obj
 0001:00003710       __ehhandler$?_Copy@?$basic_string@DU?$char_traits@D@std@@V?$allocator@D@2@@std@@QAEXII@Z 10004710 f   LinkDataScriptLibrary.obj
 0001:00003730       __unwindfunclet$?fetchFile@LinkDataScriptLibrary@U2@@SA?AVQScriptValue@@PAVQScriptContext@@PAVQScriptEngine@@@Z$0 10004730 f   LinkDataScriptLibrary.obj
 0001:00003739       __unwindfunclet$?fetchFile@LinkDataScriptLibrary@U2@@SA?AVQScriptValue@@PAVQScriptContext@@PAVQScriptEngine@@@Z$1 10004739 f   LinkDataScriptLibrary.obj
 0001:00003753       __unwindfunclet$?fetchFile@LinkDataScriptLibrary@U2@@SA?AVQScriptValue@@PAVQScriptContext@@PAVQScriptEngine@@@Z$2 10004753 f   LinkDataScriptLibrary.obj
 0001:0000375c       __unwindfunclet$?fetchFile@LinkDataScriptLibrary@U2@@SA?AVQScriptValue@@PAVQScriptContext@@PAVQScriptEngine@@@Z$3 1000475c f   LinkDataScriptLibrary.obj
 0001:00003765       __unwindfunclet$?fetchFile@LinkDataScriptLibrary@U2@@SA?AVQScriptValue@@PAVQScriptContext@@PAVQScriptEngine@@@Z$5 10004765 f   LinkDataScriptLibrary.obj
 0001:0000376e       __unwindfunclet$?fetchFile@LinkDataScriptLibrary@U2@@SA?AVQScriptValue@@PAVQScriptContext@@PAVQScriptEngine@@@Z$6 1000476e f   LinkDataScriptLibrary.obj
 0001:00003777       __unwindfunclet$?fetchFile@LinkDataScriptLibrary@U2@@SA?AVQScriptValue@@PAVQScriptContext@@PAVQScriptEngine@@@Z$8 10004777 f   LinkDataScriptLibrary.obj
 0001:00003780       __unwindfunclet$?fetchFile@LinkDataScriptLibrary@U2@@SA?AVQScriptValue@@PAVQScriptContext@@PAVQScriptEngine@@@Z$9 10004780 f   LinkDataScriptLibrary.obj
 0001:00003789       __unwindfunclet$?fetchFile@LinkDataScriptLibrary@U2@@SA?AVQScriptValue@@PAVQScriptContext@@PAVQScriptEngine@@@Z$10 10004789 f   LinkDataScriptLibrary.obj
 0001:00003792       __unwindfunclet$?fetchFile@LinkDataScriptLibrary@U2@@SA?AVQScriptValue@@PAVQScriptContext@@PAVQScriptEngine@@@Z$11 10004792 f   LinkDataScriptLibrary.obj
 0001:0000379b       __unwindfunclet$?fetchFile@LinkDataScriptLibrary@U2@@SA?AVQScriptValue@@PAVQScriptContext@@PAVQScriptEngine@@@Z$12 1000479b f   LinkDataScriptLibrary.obj
 0001:000037a4       __unwindfunclet$?fetchFile@LinkDataScriptLibrary@U2@@SA?AVQScriptValue@@PAVQScriptContext@@PAVQScriptEngine@@@Z$13 100047a4 f   LinkDataScriptLibrary.obj
 0001:000037ad       __unwindfunclet$?fetchFile@LinkDataScriptLibrary@U2@@SA?AVQScriptValue@@PAVQScriptContext@@PAVQScriptEngine@@@Z$14 100047ad f   LinkDataScriptLibrary.obj
 0001:000037b6       __unwindfunclet$?fetchFile@LinkDataScriptLibrary@U2@@SA?AVQScriptValue@@PAVQScriptContext@@PAVQScriptEngine@@@Z$15 100047b6 f   LinkDataScriptLibrary.obj
 0001:000037bf       __unwindfunclet$?fetchFile@LinkDataScriptLibrary@U2@@SA?AVQScriptValue@@PAVQScriptContext@@PAVQScriptEngine@@@Z$16 100047bf f   LinkDataScriptLibrary.obj
 0001:000037c8       __unwindfunclet$?fetchFile@LinkDataScriptLibrary@U2@@SA?AVQScriptValue@@PAVQScriptContext@@PAVQScriptEngine@@@Z$17 100047c8 f   LinkDataScriptLibrary.obj
 0001:000037d1       __unwindfunclet$?fetchFile@LinkDataScriptLibrary@U2@@SA?AVQScriptValue@@PAVQScriptContext@@PAVQScriptEngine@@@Z$18 100047d1 f   LinkDataScriptLibrary.obj
 0001:000037d9       __unwindfunclet$?fetchFile@LinkDataScriptLibrary@U2@@SA?AVQScriptValue@@PAVQScriptContext@@PAVQScriptEngine@@@Z$21 100047d9 f   LinkDataScriptLibrary.obj
 0001:000037e2       __unwindfunclet$?fetchFile@LinkDataScriptLibrary@U2@@SA?AVQScriptValue@@PAVQScriptContext@@PAVQScriptEngine@@@Z$22 100047e2 f   LinkDataScriptLibrary.obj
 0001:000037eb       __unwindfunclet$?fetchFile@LinkDataScriptLibrary@U2@@SA?AVQScriptValue@@PAVQScriptContext@@PAVQScriptEngine@@@Z$23 100047eb f   LinkDataScriptLibrary.obj
 0001:000037f4       __unwindfunclet$?fetchFile@LinkDataScriptLibrary@U2@@SA?AVQScriptValue@@PAVQScriptContext@@PAVQScriptEngine@@@Z$24 100047f4 f   LinkDataScriptLibrary.obj
 0001:000037fd       __unwindfunclet$?fetchFile@LinkDataScriptLibrary@U2@@SA?AVQScriptValue@@PAVQScriptContext@@PAVQScriptEngine@@@Z$25 100047fd f   LinkDataScriptLibrary.obj
 0001:00003806       __unwindfunclet$?fetchFile@LinkDataScriptLibrary@U2@@SA?AVQScriptValue@@PAVQScriptContext@@PAVQScriptEngine@@@Z$26 10004806 f   LinkDataScriptLibrary.obj
 0001:0000380f       __unwindfunclet$?fetchFile@LinkDataScriptLibrary@U2@@SA?AVQScriptValue@@PAVQScriptContext@@PAVQScriptEngine@@@Z$27 1000480f f   LinkDataScriptLibrary.obj
 0001:00003818       __unwindfunclet$?fetchFile@LinkDataScriptLibrary@U2@@SA?AVQScriptValue@@PAVQScriptContext@@PAVQScriptEngine@@@Z$28 10004818 f   LinkDataScriptLibrary.obj
 0001:00003821       __unwindfunclet$?fetchFile@LinkDataScriptLibrary@U2@@SA?AVQScriptValue@@PAVQScriptContext@@PAVQScriptEngine@@@Z$7 10004821 f   LinkDataScriptLibrary.obj
 0001:0000382a       __unwindfunclet$?fetchFile@LinkDataScriptLibrary@U2@@SA?AVQScriptValue@@PAVQScriptContext@@PAVQScriptEngine@@@Z$4 1000482a f   LinkDataScriptLibrary.obj
 0001:00003833       __ehhandler$?fetchFile@LinkDataScriptLibrary@U2@@SA?AVQScriptValue@@PAVQScriptContext@@PAVQScriptEngine@@@Z 10004833 f   LinkDataScriptLibrary.obj
 0001:00003860       __unwindfunclet$?init@LinkDataScriptLibrary@U2@@SAXPAVWorkflowScriptEngine@2@@Z$0 10004860 f   LinkDataScriptLibrary.obj
 0001:00003869       __unwindfunclet$?init@LinkDataScriptLibrary@U2@@SAXPAVWorkflowScriptEngine@2@@Z$1 10004869 f   LinkDataScriptLibrary.obj
 0001:00003872       __unwindfunclet$?init@LinkDataScriptLibrary@U2@@SAXPAVWorkflowScriptEngine@2@@Z$2 10004872 f   LinkDataScriptLibrary.obj
 0001:0000387b       __unwindfunclet$?init@LinkDataScriptLibrary@U2@@SAXPAVWorkflowScriptEngine@2@@Z$3 1000487b f   LinkDataScriptLibrary.obj
 0001:00003884       __unwindfunclet$?init@LinkDataScriptLibrary@U2@@SAXPAVWorkflowScriptEngine@2@@Z$4 10004884 f   LinkDataScriptLibrary.obj
 0001:0000388d       __unwindfunclet$?init@LinkDataScriptLibrary@U2@@SAXPAVWorkflowScriptEngine@2@@Z$5 1000488d f   LinkDataScriptLibrary.obj
 0001:00003896       __unwindfunclet$?init@LinkDataScriptLibrary@U2@@SAXPAVWorkflowScriptEngine@2@@Z$6 10004896 f   LinkDataScriptLibrary.obj
 0001:0000389f       __unwindfunclet$?init@LinkDataScriptLibrary@U2@@SAXPAVWorkflowScriptEngine@2@@Z$7 1000489f f   LinkDataScriptLibrary.obj
 0001:000038a8       __unwindfunclet$?init@LinkDataScriptLibrary@U2@@SAXPAVWorkflowScriptEngine@2@@Z$9 100048a8 f   LinkDataScriptLibrary.obj
 0001:000038b1       __ehhandler$?init@LinkDataScriptLibrary@U2@@SAXPAVWorkflowScriptEngine@2@@Z 100048b1 f   LinkDataScriptLibrary.obj
 0001:000038d0       __unwindfunclet$?onProxyAuthenticationRequired@LinkDataRequestHandler@U2@@AAEXABVQNetworkProxy@@PAVQAuthenticator@@@Z$0 100048d0 f   LinkDataScriptLibrary.obj
 0001:000038d9       __unwindfunclet$?onProxyAuthenticationRequired@LinkDataRequestHandler@U2@@AAEXABVQNetworkProxy@@PAVQAuthenticator@@@Z$1 100048d9 f   LinkDataScriptLibrary.obj
 0001:000038e2       __ehhandler$?onProxyAuthenticationRequired@LinkDataRequestHandler@U2@@AAEXABVQNetworkProxy@@PAVQAuthenticator@@@Z 100048e2 f   LinkDataScriptLibrary.obj
 0001:00003900       __unwindfunclet$?readScript@U2@@YA?AVQString@@ABV2@@Z$0 10004900 f   LinkDataScriptLibrary.obj
 0001:00003909       __unwindfunclet$?readScript@U2@@YA?AVQString@@ABV2@@Z$1 10004909 f   LinkDataScriptLibrary.obj
 0001:00003912       __unwindfunclet$?readScript@U2@@YA?AVQString@@ABV2@@Z$2 10004912 f   LinkDataScriptLibrary.obj
 0001:0000392c       __ehhandler$?readScript@U2@@YA?AVQString@@ABV2@@Z 1000492c f   LinkDataScriptLibrary.obj
 0001:00003950       __unwindfunclet$?sl_onReplyFinished@LinkDataRequestHandler@U2@@AAEXPAVQNetworkReply@@@Z$0 10004950 f   LinkDataScriptLibrary.obj
 0001:00003959       __unwindfunclet$?sl_onReplyFinished@LinkDataRequestHandler@U2@@AAEXPAVQNetworkReply@@@Z$1 10004959 f   LinkDataScriptLibrary.obj
 0001:00003962       __ehhandler$?sl_onReplyFinished@LinkDataRequestHandler@U2@@AAEXPAVQNetworkReply@@@Z 10004962 f   LinkDataScriptLibrary.obj
 0001:00003980       __unwindfunclet$??0LinkDataSupportPlugin@U2@@QAE@XZ$0 10004980 f   LinkDataSupportPlugin.obj
 0001:00003989       __unwindfunclet$??0LinkDataSupportPlugin@U2@@QAE@XZ$1 10004989 f   LinkDataSupportPlugin.obj
 0001:00003992       __unwindfunclet$??0LinkDataSupportPlugin@U2@@QAE@XZ$2 10004992 f   LinkDataSupportPlugin.obj
 0001:0000399b       __ehhandler$??0LinkDataSupportPlugin@U2@@QAE@XZ 1000499b f   LinkDataSupportPlugin.obj
 0001:000039c0       ??__F?_Generic_object@?$_Error_objects@H@std@@2V_Generic_error_category@2@A@@YAXXZ 100049c0 f   LinkDataScriptLibrary.obj
 0001:000039d0       ??__F?_Iostream_object@?$_Error_objects@H@std@@2V_Iostream_error_category@2@A@@YAXXZ 100049d0 f   LinkDataScriptLibrary.obj
 0001:000039e0       ??__F?_System_object@?$_Error_objects@H@std@@2V_System_error_category@2@A@@YAXXZ 100049e0 f   LinkDataScriptLibrary.obj
 0001:000039f0       ??__FLINKDATA_API_URL@U2@@YAXXZ 100049f0 f   LinkDataScriptLibrary.obj
 0001:00003a00       ??__FLINKDATA_OBJ_NAME@U2@@YAXXZ 10004a00 f   LinkDataScriptLibrary.obj
 0001:00003a10       ??__FLINKDATA_USERDATA_OBJ_NAME@U2@@YAXXZ 10004a10 f   LinkDataScriptLibrary.obj
 0001:00003a20       ??__FalgoLog@U2@@YAXXZ     10004a20 f   LinkDataScriptLibrary.obj
 0001:00003a30       ??__FcmdLog@U2@@YAXXZ      10004a30 f   LinkDataScriptLibrary.obj
 0001:00003a40       ??__FcoreLog@U2@@YAXXZ     10004a40 f   LinkDataScriptLibrary.obj
 0001:00003a50       ??__FioLog@U2@@YAXXZ       10004a50 f   LinkDataScriptLibrary.obj
 0001:00003a60       ??__FperfLog@U2@@YAXXZ     10004a60 f   LinkDataScriptLibrary.obj
 0001:00003a70       ??__FscriptLog@U2@@YAXXZ   10004a70 f   LinkDataScriptLibrary.obj
 0001:00003a80       ??__FtaskLog@U2@@YAXXZ     10004a80 f   LinkDataScriptLibrary.obj
 0001:00003a90       ??__FuiLog@U2@@YAXXZ       10004a90 f   LinkDataScriptLibrary.obj
 0001:00003aa0       ??__FuserActLog@U2@@YAXXZ  10004aa0 f   LinkDataScriptLibrary.obj
 0001:00003ab0       ??__F?_Generic_object@?$_Error_objects@H@std@@2V_Generic_error_category@2@A@@YAXXZ 10004ab0 f   LinkDataSupportPlugin.obj
 0001:00003ac0       ??__F?_Iostream_object@?$_Error_objects@H@std@@2V_Iostream_error_category@2@A@@YAXXZ 10004ac0 f   LinkDataSupportPlugin.obj
 0001:00003ad0       ??__F?_System_object@?$_Error_objects@H@std@@2V_System_error_category@2@A@@YAXXZ 10004ad0 f   LinkDataSupportPlugin.obj
 0001:00003ae0       ??__F?_Generic_object@?$_Error_objects@H@std@@2V_Generic_error_category@2@A@@YAXXZ 10004ae0 f   moc_LinkDataScriptLibrary.obj
 0001:00003af0       ??__F?_Iostream_object@?$_Error_objects@H@std@@2V_Iostream_error_category@2@A@@YAXXZ 10004af0 f   moc_LinkDataScriptLibrary.obj
 0001:00003b00       ??__F?_System_object@?$_Error_objects@H@std@@2V_System_error_category@2@A@@YAXXZ 10004b00 f   moc_LinkDataScriptLibrary.obj
 0001:00003b10       ??__F?_Generic_object@?$_Error_objects@H@std@@2V_Generic_error_category@2@A@@YAXXZ 10004b10 f   moc_LinkDataSupportPlugin.obj
 0001:00003b20       ??__F?_Iostream_object@?$_Error_objects@H@std@@2V_Iostream_error_category@2@A@@YAXXZ 10004b20 f   moc_LinkDataSupportPlugin.obj
 0001:00003b30       ??__F?_System_object@?$_Error_objects@H@std@@2V_System_error_category@2@A@@YAXXZ 10004b30 f   moc_LinkDataSupportPlugin.obj
 0001:00003b40       ??__Fdummy@?A0x896ef0f2@@YAXXZ 10004b40 f   qrc_linkdata_support.obj
 0002:0000021c       _algoLog$initializer$      1000521c     LinkDataScriptLibrary.obj
 0002:00000220       _cmdLog$initializer$       10005220     LinkDataScriptLibrary.obj
 0002:00000224       _coreLog$initializer$      10005224     LinkDataScriptLibrary.obj
 0002:00000228       _ioLog$initializer$        10005228     LinkDataScriptLibrary.obj
 0002:0000022c       _perfLog$initializer$      1000522c     LinkDataScriptLibrary.obj
 0002:00000230       _scriptLog$initializer$    10005230     LinkDataScriptLibrary.obj
 0002:00000234       _taskLog$initializer$      10005234     LinkDataScriptLibrary.obj
 0002:00000238       _uiLog$initializer$        10005238     LinkDataScriptLibrary.obj
 0002:0000023c       _userActLog$initializer$   1000523c     LinkDataScriptLibrary.obj
 0002:00000240       _LINKDATA_API_URL$initializer$ 10005240     LinkDataScriptLibrary.obj
 0002:00000244       _LINKDATA_OBJ_NAME$initializer$ 10005244     LinkDataScriptLibrary.obj
 0002:00000248       _LINKDATA_USERDATA_OBJ_NAME$initializer$ 10005248     LinkDataScriptLibrary.obj
 0002:0000024c       ?_Generic_object$initializer$@?$_Error_objects@H@std@@2P6AXXZA 1000524c     LinkDataScriptLibrary.obj
 0002:00000250       ?_Iostream_object$initializer$@?$_Error_objects@H@std@@2P6AXXZA 10005250     LinkDataScriptLibrary.obj
 0002:00000254       ?_System_object$initializer$@?$_Error_objects@H@std@@2P6AXXZA 10005254     LinkDataScriptLibrary.obj
 0002:00000258       ?staticMetaObject$initializer$@LinkDataRequestHandler@U2@@2P6AXXZA 10005258     moc_LinkDataScriptLibrary.obj
 0002:0000025c       ?staticMetaObject$initializer$@LinkDataSupportPlugin@U2@@2P6AXXZA 1000525c     moc_LinkDataSupportPlugin.obj
 0002:00000260       _dummy$initializer$        10005260     qrc_linkdata_support.obj
 0002:0000026c       _pcinit                    1000526c     MSVCRT:crtdll.obj
 0002:00000270       _pinit                     10005270     MSVCRT:atonexit.obj
 0002:00000638       _qt_meta_stringdata_U2__LinkDataRequestHandler 10005638     moc_LinkDataScriptLibrary.obj
 0002:00000738       _qt_meta_data_U2__LinkDataRequestHandler 10005738     moc_LinkDataScriptLibrary.obj
 0002:000007bc       _qt_meta_stringdata_U2__LinkDataSupportPlugin 100057bc     moc_LinkDataSupportPlugin.obj
 0002:000007e8       _qt_meta_data_U2__LinkDataSupportPlugin 100057e8     moc_LinkDataSupportPlugin.obj
 0002:00000828       _qt_resource_data          10005828     qrc_linkdata_support.obj
 0002:00000ff8       _qt_resource_name          10005ff8     qrc_linkdata_support.obj
 0002:00001080       _qt_resource_struct        10006080     qrc_linkdata_support.obj
 0002:000010e4       _GS_ExceptionPointers      100060e4     MSVCRT:gs_report.obj
 0002:00001538       __catchsym$?_Copy@?$basic_string@DU?$char_traits@D@std@@V?$allocator@D@2@@std@@QAEXII@Z$5 10006538     LinkDataScriptLibrary.obj
 0002:00001548       __catchsym$?_Copy@?$basic_string@DU?$char_traits@D@std@@V?$allocator@D@2@@std@@QAEXII@Z$4 10006548     LinkDataScriptLibrary.obj
 0002:00001558       __unwindtable$?_Copy@?$basic_string@DU?$char_traits@D@std@@V?$allocator@D@2@@std@@QAEXII@Z 10006558     LinkDataScriptLibrary.obj
 0002:00001578       __ehfuncinfo$?_Copy@?$basic_string@DU?$char_traits@D@std@@V?$allocator@D@2@@std@@QAEXII@Z 10006578     LinkDataScriptLibrary.obj
 0002:0000159c       __tryblocktable$?_Copy@?$basic_string@DU?$char_traits@D@std@@V?$allocator@D@2@@std@@QAEXII@Z 1000659c     LinkDataScriptLibrary.obj
 0002:000015c4       __unwindtable$??H@YA?BVQByteArray@@ABV0@PBD@Z 100065c4     LinkDataScriptLibrary.obj
 0002:000015d4       __ehfuncinfo$??H@YA?BVQByteArray@@ABV0@PBD@Z 100065d4     LinkDataScriptLibrary.obj
 0002:000015f8       __unwindtable$??H@YA?BVQByteArray@@PBDABV0@@Z 100065f8     LinkDataScriptLibrary.obj
 0002:00001608       __ehfuncinfo$??H@YA?BVQByteArray@@PBDABV0@@Z 10006608     LinkDataScriptLibrary.obj
 0002:0000162c       __unwindtable$??__EalgoLog@U2@@YAXXZ 1000662c     LinkDataScriptLibrary.obj
 0002:00001634       __ehfuncinfo$??__EalgoLog@U2@@YAXXZ 10006634     LinkDataScriptLibrary.obj
 0002:00001658       __unwindtable$??__EcmdLog@U2@@YAXXZ 10006658     LinkDataScriptLibrary.obj
 0002:00001660       __ehfuncinfo$??__EcmdLog@U2@@YAXXZ 10006660     LinkDataScriptLibrary.obj
 0002:00001684       __unwindtable$??__EcoreLog@U2@@YAXXZ 10006684     LinkDataScriptLibrary.obj
 0002:0000168c       __ehfuncinfo$??__EcoreLog@U2@@YAXXZ 1000668c     LinkDataScriptLibrary.obj
 0002:000016b0       __unwindtable$??__EioLog@U2@@YAXXZ 100066b0     LinkDataScriptLibrary.obj
 0002:000016b8       __ehfuncinfo$??__EioLog@U2@@YAXXZ 100066b8     LinkDataScriptLibrary.obj
 0002:000016dc       __unwindtable$??__EperfLog@U2@@YAXXZ 100066dc     LinkDataScriptLibrary.obj
 0002:000016e4       __ehfuncinfo$??__EperfLog@U2@@YAXXZ 100066e4     LinkDataScriptLibrary.obj
 0002:00001708       __unwindtable$??__EscriptLog@U2@@YAXXZ 10006708     LinkDataScriptLibrary.obj
 0002:00001710       __ehfuncinfo$??__EscriptLog@U2@@YAXXZ 10006710     LinkDataScriptLibrary.obj
 0002:00001734       __unwindtable$??__EtaskLog@U2@@YAXXZ 10006734     LinkDataScriptLibrary.obj
 0002:0000173c       __ehfuncinfo$??__EtaskLog@U2@@YAXXZ 1000673c     LinkDataScriptLibrary.obj
 0002:00001760       __unwindtable$??__EuiLog@U2@@YAXXZ 10006760     LinkDataScriptLibrary.obj
 0002:00001768       __ehfuncinfo$??__EuiLog@U2@@YAXXZ 10006768     LinkDataScriptLibrary.obj
 0002:0000178c       __unwindtable$??__EuserActLog@U2@@YAXXZ 1000678c     LinkDataScriptLibrary.obj
 0002:00001794       __ehfuncinfo$??__EuserActLog@U2@@YAXXZ 10006794     LinkDataScriptLibrary.obj
 0002:000017b8       __ehfuncinfo$?init@LinkDataScriptLibrary@U2@@SAXPAVWorkflowScriptEngine@2@@Z 100067b8     LinkDataScriptLibrary.obj
 0002:000017dc       __unwindtable$?init@LinkDataScriptLibrary@U2@@SAXPAVWorkflowScriptEngine@2@@Z 100067dc     LinkDataScriptLibrary.obj
 0002:0000182c       __ehfuncinfo$?fetchFile@LinkDataScriptLibrary@U2@@SA?AVQScriptValue@@PAVQScriptContext@@PAVQScriptEngine@@@Z 1000682c     LinkDataScriptLibrary.obj
 0002:00001850       __unwindtable$?fetchFile@LinkDataScriptLibrary@U2@@SA?AVQScriptValue@@PAVQScriptContext@@PAVQScriptEngine@@@Z 10006850     LinkDataScriptLibrary.obj
 0002:00001990       __unwindtable$??0LinkDataRequestHandler@U2@@QAE@PAVQEventLoop@@@Z 10006990     LinkDataScriptLibrary.obj
 0002:000019a0       __ehfuncinfo$??0LinkDataRequestHandler@U2@@QAE@PAVQEventLoop@@@Z 100069a0     LinkDataScriptLibrary.obj
 0002:000019c4       __unwindtable$?sl_onReplyFinished@LinkDataRequestHandler@U2@@AAEXPAVQNetworkReply@@@Z 100069c4     LinkDataScriptLibrary.obj
 0002:000019d4       __ehfuncinfo$?sl_onReplyFinished@LinkDataRequestHandler@U2@@AAEXPAVQNetworkReply@@@Z 100069d4     LinkDataScriptLibrary.obj
 0002:000019f8       __unwindtable$?onProxyAuthenticationRequired@LinkDataRequestHandler@U2@@AAEXABVQNetworkProxy@@PAVQAuthenticator@@@Z 100069f8     LinkDataScriptLibrary.obj
 0002:00001a08       __ehfuncinfo$?onProxyAuthenticationRequired@LinkDataRequestHandler@U2@@AAEXABVQNetworkProxy@@PAVQAuthenticator@@@Z 10006a08     LinkDataScriptLibrary.obj
 0002:00001a2c       __unwindtable$??1LinkDataRequestHandler@U2@@UAE@XZ 10006a2c     LinkDataScriptLibrary.obj
 0002:00001a3c       __ehfuncinfo$??1LinkDataRequestHandler@U2@@UAE@XZ 10006a3c     LinkDataScriptLibrary.obj
 0002:00001a60       __unwindtable$??_GLinkDataRequestHandler@U2@@UAEPAXI@Z 10006a60     LinkDataScriptLibrary.obj
 0002:00001a70       __ehfuncinfo$??_GLinkDataRequestHandler@U2@@UAEPAXI@Z 10006a70     LinkDataScriptLibrary.obj
 0002:00001a94       __unwindtable$?readScript@U2@@YA?AVQString@@ABV2@@Z 10006a94     LinkDataScriptLibrary.obj
 0002:00001aac       __ehfuncinfo$?readScript@U2@@YA?AVQString@@ABV2@@Z 10006aac     LinkDataScriptLibrary.obj
 0002:00001ad0       __ehfuncinfo$??0LinkDataSupportPlugin@U2@@QAE@XZ 10006ad0     LinkDataSupportPlugin.obj
 0002:00001af4       __unwindtable$??0LinkDataSupportPlugin@U2@@QAE@XZ 10006af4     LinkDataSupportPlugin.obj
 0002:00001b20       __sehtable$__onexit        10006b20     MSVCRT:atonexit.obj
 0002:00001b40       __sehtable$___DllMainCRTStartup 10006b40     MSVCRT:crtdll.obj
 0002:00001b68       __sehtable$??_M@YGXPAXIHP6EX0@Z@Z 10006b68     MSVCRT:ehvecdtr.obj
 0002:00001b88       __sehtable$?__ArrayUnwind@@YGXPAXIHP6EX0@Z@Z 10006b88     MSVCRT:ehvecdtr.obj
 0002:00001ba8       __sehtable$__IsNonwritableInCurrentImage 10006ba8     MSVCRT:pesect.obj
 0002:00001bd0       .edata                     10006bd0     linkdata_support.exp
 0002:00001bf8       rgpv                       10006bf8     linkdata_support.exp
 0002:00001bfc       rgszName                   10006bfc     linkdata_support.exp
 0002:00001c00       rgwOrd                     10006c00     linkdata_support.exp
 0002:00001c02       szName                     10006c02     linkdata_support.exp
 0002:00001c17       $N00001                    10006c17     linkdata_support.exp
 0002:0000210e       .idata$6                   1000710e     U2Core:U2Core.dll
 0002:00002196       .idata$6                   10007196     U2Lang:U2Lang.dll
 0002:0000242a       .idata$6                   1000742a     Qt5Script:Qt5Script.dll
 0002:0000265c       .idata$6                   1000765c     Qt5Network:Qt5Network.dll
 0002:00002dde       .idata$6                   10007dde     Qt5Core:Qt5Core.dll
 0002:00002e84       .idata$6                   10007e84     msvcprt:MSVCP120.dll
 0002:00002f08       .idata$6                   10007f08     MSVCRT:MSVCR120.dll
 0002:0000311c       .idata$6                   1000811c     kernel32:KERNEL32.dll
 0003:000001e8       __Tuple_alloc              100091e8     LinkDataScriptLibrary.obj
 0003:000001e9       _ignore                    100091e9     LinkDataScriptLibrary.obj
 0003:000001ea       _allocator_arg             100091ea     LinkDataScriptLibrary.obj
 0003:000001eb       _piecewise_construct       100091eb     LinkDataScriptLibrary.obj
 0003:000001ec       _taskLog                   100091ec     LinkDataScriptLibrary.obj
 0003:000001f4       _algoLog                   100091f4     LinkDataScriptLibrary.obj
 0003:000001fc       _userActLog                100091fc     LinkDataScriptLibrary.obj
 0003:00000204       _ioLog                     10009204     LinkDataScriptLibrary.obj
 0003:0000020c       _LINKDATA_API_URL          1000920c     LinkDataScriptLibrary.obj
 0003:00000210       _coreLog                   10009210     LinkDataScriptLibrary.obj
 0003:00000218       _uiLog                     10009218     LinkDataScriptLibrary.obj
 0003:00000220       _scriptLog                 10009220     LinkDataScriptLibrary.obj
 0003:00000228       _LINKDATA_USERDATA_OBJ_NAME 10009228     LinkDataScriptLibrary.obj
 0003:0000022c       _perfLog                   1000922c     LinkDataScriptLibrary.obj
 0003:00000234       _cmdLog                    10009234     LinkDataScriptLibrary.obj
 0003:0000023c       _LINKDATA_OBJ_NAME         1000923c     LinkDataScriptLibrary.obj
 0003:00000248       __Tuple_alloc              10009248     LinkDataSupportPlugin.obj
 0003:00000249       _ignore                    10009249     LinkDataSupportPlugin.obj
 0003:0000024a       _allocator_arg             1000924a     LinkDataSupportPlugin.obj
 0003:0000024b       _piecewise_construct       1000924b     LinkDataSupportPlugin.obj
 0003:0000024c       __Tuple_alloc              1000924c     moc_LinkDataScriptLibrary.obj
 0003:0000024d       _ignore                    1000924d     moc_LinkDataScriptLibrary.obj
 0003:0000024e       _allocator_arg             1000924e     moc_LinkDataScriptLibrary.obj
 0003:0000024f       _piecewise_construct       1000924f     moc_LinkDataScriptLibrary.obj
 0003:00000250       __Tuple_alloc              10009250     moc_LinkDataSupportPlugin.obj
 0003:00000251       _ignore                    10009251     moc_LinkDataSupportPlugin.obj
 0003:00000252       _allocator_arg             10009252     moc_LinkDataSupportPlugin.obj
 0003:00000253       _piecewise_construct       10009253     moc_LinkDataSupportPlugin.obj
 0003:00000258       ___proc_attached           10009258     MSVCRT:crtdll.obj
 0003:00000260       _GS_ExceptionRecord        10009260     MSVCRT:gs_report.obj
 0003:000002b0       _GS_ContextRecord          100092b0     MSVCRT:gs_report.obj
 0003:0000057c       _DebuggerWasPresent        1000957c     MSVCRT:gs_report.obj
 0004:00000060       $R000000                   1000a060     * linker generated manifest res *

 Exports

  ordinal    name

        1    _ugene_plugin_init
               exported name: ugene_plugin_init
